:020000040001F9
:1090000018320020C1930100C9930100CB930100E5
:10901000CD930100CF930100D19301000000000027
:10902000000000000000000000000000D3930100D9
:10903000D593010000000000D7930100D9930100EF
:1090400041970100DB930100B19A0100DB9301001D
:10905000DB9301000000000079950100DB93010023
:10906000DB930100DB930100DB930100DB93010044
:10907000DB930100DB930100DB930100DB93010034
:10908000DB93010099970100DB930100DB93010062
:10909000BD970100DB930100C1970100DB93010044
:1090A000DB930100DB9301000000000000000000E2
:1090B000DB930100DB9301000000000000000000D2
:1090C00000000000000000000000000000000000A0
:1090D0000000000000000000000000000000000090
:1090E0000000000000000000000000000000000080
:1090F0000000000000000000000000000000000070
:10910000000000000000000000000000000000005F
:10911000000000000000000000000000000000004F
:10912000000000000000000000000000000000003F
:10913000000000000000000000000000000000002F
:10914000000000000000000000000000000000001F
:10915000000000000000000000000000000000000F
:1091600000000000000000000000000000000000FF
:1091700000000000000000000000000000000000EF
:1091800000000000000000000000000000000000DF
:1091900000000000000000000000000000000000CF
:1091A00000000000000000000000000000000000BF
:1091B00000000000000000000000000000000000AF
:1091C000000000000000000000000000000000009F
:1091D000000000000000000000000000000000008F
:1091E000000000000000000000000000000000007F
:1091F000000000000000000000000000000000006F
:10920000DFF80CD000F07AF900480047FDCC0100EF
:109210001832002030B450E8012F93B2C48923449F
:109220008489A34228BF1B1B0489A34202BFBFF34A
:109230002F8F002007E0C3EA020340E80134002C2E
:10924000E9D14FF001000A6030BC704750E8012FAF
:10925000C2EA024240E801210029F7D1704730B448
:1092600050E8022F1FFAA2F3C488A34202BFBFF343
:109270002F8F00200DE0C48923448489A34228BF96
:109280001B1BC2EA034340E80234002CE8D14FF034
:1092900001000A6030BC704750E8022FC2EA224247
:1092A00040E802210029F7D17047034653E8022F16
:1092B000D988B2EB324F4FF0000017BF92B241EAAB
:1092C000014142EA014104E05A68B2EB324F08BF63
:1092D000012043E80212002AE8D1704730B4044666
:1092E00054E8000F0D4644E80053002BF8D11560F8
:1092F00030BC704730B4044654E8000F40EA010522
:1093000044E80053002BF7D1156030BC704730B4EF
:10931000044654E8000F00EA010544E80053002B1E
:10932000F7D1156030BC704730B4044654E8000FE4
:1093300080EA010544E80053002BF7D1156030BCEA
:10934000704730B4044654E8000F00EB010544E8D0
:109350000053002BF7D1156030BC704730B4044681
:1093600054E8000FA0EB010544E80053002BF7D1AF
:10937000156030BC704770B404464FF0000054E8EC
:10938000006F0D68AE4207BF44E80023012044E8A7
:1093900000630E60002B1CBF0020F0E770BC70471C
:1093A00030B4044654E8000F88422CBF451A0546E5
:1093B00044E80053002BF5D1156030BC7047000025
:1093C0000648804706480047FEE7FEE7FEE7FEE75F
:1093D000FEE7FEE7FEE7FEE7FEE7FEE7C5970100D2
:1093E000019201002DE9F05F0546002092469B4660
:1093F00088460646814640241BE0284641464746AB
:10940000224600F06BF853465A46C01A914110D3D9
:1094100011461846224600F016F82D1A67EB01088F
:109420004F4622460120002100F00DF817EB0009FD
:109430004E41201EA4F10104DFDC484631462A4695
:109440004346BDE8F09F202A04DB203A00FA02F1EF
:10945000002070479140C2F1200320FA03F3194322
:109460009040704700487047AC1E020040EA01037C
:109470009B0703D009E008C9121F08C0042AFAD2CA
:1094800003E011F8013B00F8013B521EF9D270478E
:10949000D2B201E000F8012B491EFBD27047002236
:1094A000F6E710B513460A4604461946FFF7F0FFE3
:1094B000204610BD421C10F8011B0029FBD1801A68
:1094C000704730B504460020034600E05B1C934221
:1094D00003D2E05CCD5C401BF8D030BD202A04DB19
:1094E000203A21FA02F00021704721FA02F3D0401D
:1094F000C2F120029140084319467047064C074DBF
:1095000006E0E06840F0010394E807009847103453
:10951000AC42F6D3FFF778FE84250200A4250200B2
:1095200070B58C1810F8015B15F0070301D110F825
:10953000013B2A1106D110F8012B03E010F8016B52
:1095400001F8016B5B1EF9D12B0705D40023521ED5
:109550000DD401F8013BFAE710F8013BCB1A921C3D
:1095600003E013F8015B01F8015B521EF9D5A1423B
:10957000D8D3002070BD00002DE9F04700268AB046
:10958000DFF85091B0464FF48075012437460696B7
:10959000284604F04DFC38B1D9F80403204203D02A
:1095A000284604F03BFC26432D1D64007F1CADB211
:1095B000082FEDD34FF4BE74204604F039FC48B1B7
:1095C000204604F02BFC46F0004606AA01210020AC
:1095D00004F010FC404D16F0FF0F15D001270024B9
:1095E00037420DD009EB8401D1F81005D1F81015E0
:1095F000C0F3042055F82420C1F3014102B1904783
:109600007F00641C082CEBD3002E5FDA4FF0FF3094
:10961000CDF8108054E0281910F8507F90F9000020
:1096200027F0C008401C3BD007A9404603F09FFE2E
:1096300010B34FEA9719404601F0A4FD55F8207089
:109640001FB1B9F1030F03D006E0B9F1030F27D121
:1096500004A9404603F093FE4FF0A04101EB8800BF
:10966000D0F8000706A9C0F3014A404603F07FFE88
:1096700018B1BAF1020F03D012E0BAF1030F0FD103
:10968000B9F1030F08D1BAF1020F1DD002214046F3
:1096900004F094FB761CF6B217B149464046B84731
:1096A000641C042CB7D3002E10D06A460121002080
:1096B00004F0A0FB06990098884207D00690049811
:1096C000002634460790A6E70321E0E70AB0BDE88C
:1096D000F087000000600040B021002000F01F0271
:1096E000012191404009800000F1E020C0F8801283
:1096F000704700F01F02012191404009800000F1F5
:10970000E020C0F80011704700F01F0201219140D5
:109710004009800000F1E020C0F8001270474907BE
:10972000090E002806DA00F00F0000F1E02080F8B2
:10973000141D704700F1E02080F80014704700000D
:1097400070B54FF48076304603F022FF114CB5051A
:1097500060B1304603F023FF0120C5F808036079AB
:1097600020B9012060712168002088474FF482767B
:10977000304603F00DFF00280AD0304603F00FFFFB
:109780000220C5F808032168BDE8704001200847A1
:1097900070BD0000D01B002007480021C0F8401118
:1097A000C0F84411C0F84811C0F84C11C0F80011BD
:1097B000C0F8041107F0B4BC0010014007F0FEBB74
:1097C00005F08CB8F0B5A848A74B012600781B1D02
:1097D0001A1D4FF0805106280BD11C78240708D1A0
:1097E0001478C4F30314032C06D0042C04D0052CE5
:1097F00002D0062807D011E0B1F824439B4DC4F3F2
:1098000004242C6002E01C78240707D11478C4F3E8
:109810000314032C02D1974D954C6C67D1F830514D
:10982000D1F84442944FC4F342343C6006280CD132
:109830001C78240709D11478C4F30314032C04D131
:109840008E4C276827F0807727604FF080470024F0
:10985000C7F80C41C7F81041874F3F1F3C600628EE
:1098600007D11F783F0704D11778C7F30317032FD9
:1098700002D0062808D01FE0DFF8FCC103270CF156
:10988000640CCCF8007007E01F783F0714D11778FC
:10989000C7F30317032F0FD1DFF8E4C10527CCF876
:1098A0000070774F78373E60754F08373C600CF199
:1098B000040C3F27CCF80070724F3F68DFF8C8C136
:1098C000CCF800706F4F3F1D3F680CF1040CCCF8D2
:1098D00000706C4F08373F680CF1040CCCF8007036
:1098E000684F0C373F680CF1040CCCF80070654FE2
:1098F00010373F680CF1040CCCF80070614F14373E
:109900003F680CF1040CCCF800705E4F18373F68CC
:10991000DFF874C10CF1200CCCF80070594F1C37E3
:109920003F680CF1040CCCF80070564F20373F68AC
:109930000CF1040CCCF80070524F24373F680CF146
:10994000040CCCF800704F4F28373F680CF1040C22
:10995000CCF800704B4F2C373F680CF1040CCCF85E
:109960000070484F30373F68DFF81CC10CF1400CE5
:10997000CCF80070434F34373F680CF1040CCCF83E
:109980000070404F38373F680CF1040CCCF8007081
:109990003C4F3C373F680CF1040CCCF80070394F59
:1099A00040373F680CF1040CCCF80070DFF8DCC0E5
:1099B000FB27CCF80070062813D11F783F0710D181
:1099C0001778C7F30317032F03D0042F01D0052FF7
:1099D00007D1D1F85872DFF8B8C007F04F07CCF8BC
:1099E00000702C480268D20702D06FF001020260BA
:1099F000062D08D1D1F83401062804D12648016883
:109A000041F4806101604FF01021D1F8000200287C
:109A100003DBD1F80402002822DA204A166020482D
:109A20000368002BFCD01523C1F800320568002D17
:109A3000FCD0C1F8043201680029FCD01460016830
:109A40000029FCD0BFF34F8F0C48F0380168154A4D
:109A500001F4E06111430160BFF34F8F00BFFDE7E8
:109A6000124911480860F0BDE00F00F04035014098
:109A70000DF0ADBA00C007403C050040FCED00E031
:109A8000105600400404001020C5004018F50040A6
:109A9000E40E0040000400403C17004004E5014093
:109AA00000E401400400FA050090D003E41C00200B
:109AB0000149024807F0B4BB0C22002000200040FE
:109AC00002E008C8121F08C1002AFAD17047704787
:109AD000002001E001C1121F002AFBD170470000E5
:109AE0000121202803DA81400548014003E0402895
:109AF00002DA2038814009B1012070470020704708
:109B0000FC06FFBD082806D228B1012803D004288E
:109B100001D0012070470020704710B560B159B1E5
:109B200002780B785208B2EB530F05D10622401C85
:109B3000491CFFF7C6FC08B1002010BD012010BD74
:109B4000800701D00020704701207047C3688B4216
:109B500006D811440069491E814201D8012070478E
:109B60000020704710B501220221002001F01AF9EF
:109B700008B1072810D107220221012001F012F9B3
:109B800008B1072808D100210A22084601F00AF985
:109B900008B1072800D1002010BD000010B550B159
:109BA0000A480321008801EB004009A104F026FBCC
:109BB00006F092F903E00321094800F030FC002888
:109BC00003D0BDE8104000F0CBB810BD281D002028
:109BD000457261736520626F6E647321000000003E
:109BE000541D002070B58CB015460E4600236C46FF
:109BF000C3F10F01415CE1545B1C102BF8D30D2124
:109C000004F11000FFF74BFC0020C0F10F02315CA3
:109C10002244401C11740328F7D3684646DF002015
:109C2000C0F10F01214491F820102954401C032851
:109C3000F6D30CB070BD022000F0BEBF0149097917
:109C400000F064BDA81B002070B50024064D06E09E
:109C50006868012110F8340004F01AFF641C2878A9
:109C60008442F5D3002070BDD81B0020F8B51546FE
:109C70000C460646052A01D20720F8BD05F004F877
:109C800018B904F0C9FF0028F7D1124900224E602C
:109C90000C708D60C1E90422C1E906220E4D0DE071
:109CA00006EBC4002968009181788DF801100078D6
:109CB0000A4A694604F03EFF0028DED1641EE4B281
:109CC000EED2BDE8F84004480021054A001D00F02E
:109CD00053B80000D81B0020301B020099C00100BF
:109CE00015B5010072B604F03FFB00BF04F076F931
:109CF0000028FBD1104C0121208801EB00400FA16E
:109D000004F07CFA10480068C00700D000BE20882C
:109D1000022101EB00400DA104F070FABFF34F8F58
:109D20000948E43801680D4A01F4E061114301601B
:109D3000BFF34F8F00BFFDE7281D0020466174610F
:109D40006C206572726F7200F0ED00E053797374ED
:109D5000656D207265736574000000000400FA05EB
:109D60000EB500210091CDE901106A4644F20100D0
:109D7000FFF7B8FF0EBD0000074B9B7823B12AB157
:109D800020B10068037C1BB1082070470720704792
:109D900041744261002070475022002070B506F0E7
:109DA00081FB104800240B21047044700E4D81701B
:109DB00014206C602C706C70FFF790FC072114204D
:109DC000FFF7ADFC1420FFF794FC0848046007215E
:109DD0001120FFF7A4FC0548001F0068A8600020C0
:109DE00070BD000050220020F81B00200815014023
:109DF0002DE9FC47DFF8789099F8023073B368B327
:109E0000052902D20720BDE8FC87436933B3437CB0
:109E1000012B25D0002704460025884616468DF8DC
:109E20000050684600F038F801A807F045FBC8B1BB
:109E3000012101700F4944600968C0E90218C0E9B6
:109E400004769DF8040089F801009DF8000000F0F8
:109E500047F81420FFF758FC2846D4E70820D2E73B
:109E60000F46D8E704259DF8000000F039F8F3E725
:109E700050220020041501400649897839B130B1DB
:109E8000416921B100210174022107F025B90820A0
:109E9000704700005022002030B5EFF3108172B6F9
:109EA0000D4A9468012324B10370002900D162B6E1
:109EB00030BD93604FF0E023D3F88051074C25402C
:109EC0001560C3F88041D3F8844154605A17C3F831
:109ED000842100220270E8E75C230020FC06FFBD1D
:109EE0000B498A68002A11D000280FD1EFF31080A7
:109EF00072B60B684FF0E022C2F800314B68C2F82E
:109F0000043100228A60002800D162B67047000048
:109F10005C2300202DE9F041064608680C46411CF0
:109F20004FF0A0474FF0010506D005FA00F1C7F841
:109F30000815206803F038FF6068411C02D000213A
:109F400003F029FF3168A069C1F82405607D217DF7
:109F500032680843C2F86C05D4E900123068C0F8D2
:109F60000C15C0F81425207D012815D1A068411CCE
:109F700002D0002103F00FFFE068411C05D08540AE
:109F8000C7F80855E06803F00FFFD4E90212306803
:109F9000C0F80825C0F81015BDE8F08102F00ABE2F
:109FA0002DE9F047074600888EB0804602F0FAFAA5
:109FB000824604462D4800252A460178404600F096
:109FC000BDFB7879400734D501254FF6FF7603AB0A
:109FD0002A460721504605F0E3F9010004D0404627
:109FE00006F056FC00252BE0B1463146049802F0FD
:109FF0002DFA064648450FD004460146404602F079
:10A00000BBFA4046FFF71AFE30B9404606F012FC94
:10A010004046FFF713FE48B122460721504605F09F
:10A0200035FA010003D0404606F032FC00254E45CB
:10A0300006D0404605F098FB10B1504602F09EFA5B
:10A0400002208DF81800ADF81A807879400701D504
:10A05000012000E002208DF820008DF8215006A894
:10A0600001F0CCFB0EB0BDE8F0870000A81B00207B
:10A070002DE9FC47002517880646158090F82D002D
:10A080001446894630B13A462146484600F080FBE6
:10A09000051E09D1B0784FF00C0A18B32088C846C5
:10A0A000001DB84202D95046BDE8FC87684679DFFA
:10A0B0000028F9D12088032108F8001020881921F0
:10A0C000401C80B2208008F800102088401C80B21C
:10A0D000208000EB0801BDF8000007F01BF9218883
:10A0E00008442080F0780222C8B1218896F9033014
:10A0F00001F1030C4846BC45D5D8425421884FF0A5
:10A10000010C491C89B2218000F801C02188491C3A
:10A1100089B2218009F801302088401C20807068B5
:10A12000B8B1218890F9003001F1030C4846BC45D4
:10A13000B9D8425421880A22491C89B2218042544C
:10A140002188491C89B2218009F801302088401CEF
:10A150002080308950B1CDE900474B4606220221CC
:10A1600006F1080007F0C0F9051E9DD1308A50B1F4
:10A17000CDE900474B460722032106F1100007F006
:10A18000B3F9051E90D1308B50B1CDE900474B4655
:10A190001522142106F1180007F0A6F9051E83D137
:10A1A000306A30B13B462246494601F0A6F8051E0A
:10A1B000DBD1706A30B13B462246494602F092FE3E
:10A1C000051ED2D196F82C0038B13B4622464946AE
:10A1D000304606F0F9FB051EC7D1307838B13B4652
:10A1E00022464946304602F003FF051EBDD12846EF
:10A1F0005AE718B504460020ADF8000013466A4639
:10A20000204600F006F8002802D0BDF800002044E7
:10A2100018BD70B588B182B10024158803E0065DD1
:10A22000641C3444A4B2A54203D8061976789E4231
:10A2300001D08C42F3D38C4201D3002070BDA11C0D
:10A240001180005D401E80B270BD80F830107047F4
:10A250002DE9F0410D00044606D02CB195F87A00A6
:10A260000026012803D006E00E20BDE8F08195F815
:10A270009800012829D0D5F8A000042825D0D5F8C9
:10A280009C00042821D04FF00108A6702C2205F173
:10A290007801201DFFF7EAF884F83060D5F8A400B3
:10A2A0006063D5F8A800A0634FF6FF70A4F8A8007B
:10A2B00004F19400C4F8A400C4F8AA60A4F8AE6045
:10A2C00084F8B060207810B104E00720CDE7FF20CB
:10A2D00084F8540004F155011F27C4F89410A4F821
:10A2E000987004F198022846FFF7C2FE0028BCD1FE
:10A2F00015F13C0F0ED004F17401C4F89C10A4F8C1
:10A30000A07004F1A00205F13C00FFF7B1FE0028A7
:10A31000ABD103E0C4F89C60A4F8A06084F851803D
:10A32000208BA4F8480084F83C80266484F85060B0
:10A3300060696064454604F13C02002104F1540068
:10A3400072DF002891D125708FE710B50288102A9E
:10A350001BD0112A20D0262A1DD1007A0C460128B4
:10A3600001D0022817D1A0780521401CB0FBF1F2E2
:10A3700001FB1201204600F052F800280BD0A16B1F
:10A38000002908D0BDE810400847C27B012A02D14D
:10A390008088A1F8A80010BD0C46002184F8B210F6
:10A3A0008088B4F8A8108842F5D120790028F2D12D
:10A3B0000121DFE710B50C46022801D0032810D197
:10A3C000607800280DD000206070A178204600F051
:10A3D00026F8002805D0A16B002902D0BDE8104066
:10A3E000084710BD10B5044690F8540074DF0120F2
:10A3F00084F8B200002084F8B40084F850000621EC
:10A40000204601F001FC002808D1A178204600F088
:10A4100006F810B1A16B01B18847002010BD2DE9ED
:10A42000F05F044600780F4638B1A770002003F0B3
:10A43000F3FA012620B16670F4E00820BDE8F09F31
:10A440000025C4F8AA50A4F8AE5084F8B050A07902
:10A4500010B1A078012806D0E07968B1A078012871
:10A4600001D0022808D1616B21B184F8B1600820C5
:10A47000884701E084F8B15004F1AB0100200A5C88
:10A480000AB1304603E0401C0628F8D300204FF004
:10A4900002084FF0030A4FF0040B012F06D0022FE1
:10A4A0000CD0032F0FD0042F15D110E0A17929B1C2
:10A4B00094F8241011B908B130460DE0E17911B1DA
:10A4C00008B1404608E0207A08B1504604E0607ABE
:10A4D00008B1584600E02846A070616B41B10328DE
:10A4E00001D0042804D1607910B194F8B200A0B171
:10A4F00084F8B35004F13C0018210746FEF7CFFF63
:10A5000004F12C0084F83C60814605F059FA58B1FA
:10A5100094F82C0084F8510008E084F8B45084F8D2
:10A52000B36007208847E5E784F8516094F8240079
:10A5300050B1484605F044FA20B194F8280084F858
:10A54000520001E084F8526084F85050A27804F17F
:10A55000AA0104F19409052A4DD2DFE802F065034F
:10A560000F1B320084F83160C4F8A450C4E9101500
:10A5700084F83C808020A4F848003EE084F83180D4
:10A5800087F800A0228ABA81C4F8A4507960E168F3
:10A59000B96032E06069B860208BB8813D4684F8CC
:10A5A0003C60204606F064FF40B185F81480042129
:10A5B000204601F029FBF0B9052115E084F831A00F
:10A5C00017E0E069B860208CB8813D4684F83C60B3
:10A5D000204606F04DFF50B185F814800421204636
:10A5E00001F012FB38B9062184F8311001E084F83B
:10A5F00031B0C4F8A490A07878B13A4604F1540080
:10A60000D4F8A41072DF00287FF418AF94F830104B
:10A6100094F8540073DF0028F6D1616B11B194F8FF
:10A6200031008847002009E784F83150F5E7000041
:10A6300070B5040012D001461C221448FEF716FF24
:10A640001248134D0560206850B17ADF002806D10A
:10A650002068016829604068686005E00E2070BDD0
:10A660000B487BDF0028FAD108484FF6FF711438F9
:10A67000084A20F8041B0549343901600021FFF71E
:10A680007BFB0028EBD0032070BD0000AC1E002037
:10A69000681B00200914020010B5044600F06EF893
:10A6A000002805D02146BDE81040024802F0C3BD95
:10A6B00010BD0000D81E002070B515460E46044699
:10A6C00006F0E2FE002809D0054800EB840080690E
:10A6D0002A463146BDE8704001F0D4BA70BD000092
:10A6E000C81E002010B5002400F048F800B1012475
:10A6F000204610BD10B51821034802F077FD182838
:10A7000000D0C0B210BD0000C81E002070B50546C4
:10A710000C46084606F0B8FE60B1284600F02EF858
:10A7200040B10548294600EB8400BDE87040183070
:10A7300002F081BD002070BDC81E002070B5054626
:10A7400014460E46084606F09FFE002812D0284602
:10A7500000F014F800280DD00748294600EB8600C9
:10A7600018301CB1BDE8704002F070BDBDE870400B
:10A7700002F021BD70BD0000C81E0020142801D3C6
:10A78000002070470146014802F055BDCC1E002054
:10A790007CB5054608880C460930904201D90C204A
:10A7A0007CBD68466DDF0028FAD1218808206854F6
:10A7B00020881B21401C80B2208029542088401C06
:10A7C00080B220802844DDF801100160BDF805103A
:10A7D00081802088801D80B220809DF8001049086B
:10A7E00000D0012129542088401C208000207CBDFD
:10A7F00038B502880446212A2CD00EDC1C484FF0C4
:10A800000301102A008801EB00400ED0112A2AD142
:10A81000BDE8384017A103F0F1BC3B2A24D0562AEA
:10A8200021D18088132176DF0EE016A103F0E6FC2B
:10A83000072000F0D9FA08B1FFF792FA1448A1886E
:10A840000180144802F02CFE00280CD0BDE83840EE
:10A85000FFF786BA00200090A08869468FDF0028A5
:10A8600001D0FFF77DFA38BD8088132176DFEBE752
:10A87000281D0020446973636F6E6E6563746564A0
:10A880002E000000436F6E6E65637465642E0000D9
:10A89000481B0020481D002010B51A4C0188606834
:10A8A00010290ED011292BD1401E606028D1FFF74E
:10A8B00059F9002824D02168002921D0BDE8104092
:10A8C0000847D0B900210122084600F06BFA08B110
:10A8D00007280FD107220221012000F063FA08B1F6
:10A8E000072807D104220221002000F05BFA20B1E2
:10A8F000072802D0216801B188476068401C606069
:10A9000010BD0000601B00202DE9F04701883B4E80
:10A9100040F2F3194FF6FF7510291BD011293ED0D4
:10A92000122954D0502946D1C188F289841D914200
:10A9300041D1618902293ED18688304601F0DEFE90
:10A94000050038D004F10C0000F0F2F8A8B3294655
:10A9500030464EE0C17B8788044601292BD1A846AA
:10A96000284601F0CBFE050017D02F80002028726A
:10A97000234843464A460168C5F80A104068C5F8AE
:10A980000E0004F1100105F10A0001F083FF687266
:10A99000F08900280FD129462AE0042013E080889E
:10A9A00001F0ACFE040006D06068FFF765FA08B15C
:10A9B00005F052FF2580BDE8F087FFE76868FFF7E4
:10A9C0005BFA0028F7D0BDE8F04705F045BF87885F
:10A9D0000646384601F092FE0400ECD02B464A466B
:10A9E00006F1080104F10A0001F054FF60722146EB
:10A9F0003846BDE8F04700F0C7BC0000AC1E0020A0
:10AA0000681B00202DE9F04F0746858802883D48E5
:10AA1000012197B08346102A09D0112A49D01A2A59
:10AA20006CD1387AB1EB101F45D2012244E0354C8D
:10AA3000083CA068C0430B9061680BA802F01FFCA3
:10AA40000B990CA800F03AFC2C220CA96846FEF7E2
:10AA50000DFD0026E946A04610E000BF09EB4600C8
:10AA60005FF00004B0F804A008EB84005146001D1C
:10AA700002F0A1FB641C1D2CF6D3761C0098B0429A
:10AA8000ECD8142D05D317B00420BDE8F04FFFF724
:10AA900067B92946584602F0D9FB294608F1040057
:10AAA00002F0D4FBF87B012828D016482946001D67
:10AAB00015E029461AE000220221B1EB101F01D255
:10AAC000012600E000260F49083901F11000041D9D
:10AAD000294682B102F0BAFB36B12946204617B0AA
:10AAE000BDE8F04F02F0B2BB2946204617B0BDE8E2
:10AAF000F04F02F060BB02F05EFBF5E717B0BDE877
:10AB0000F08F0000D01E002010B5044607480078E2
:10AB100000280AD0204601F01FFC204605F0ACFFBB
:10AB20002046BDE8104001F0B9B910BD981B0020C7
:10AB3000007800F0010070470149085C7047000090
:10AB4000E81902000649095C4FF0A040D0F8100552
:10AB5000C84010F0010000D0012080F001007047D3
:10AB6000E81902002DE9FC410646C0074FF0000538
:10AB70000ED0104F00240122385D009500231146AD
:10AB8000019503F0C9F8641C042CF4D300F046F8D6
:10AB9000B0070DD5074E0024361D0022305D03237B
:10ABA00000951146019503F0B7F8641C042CF4D30A
:10ABB000BDE8FC81E419020007490B5C4FF0A0419D
:10ABC000D1F804250120984020EA0203C1F8083595
:10ABD0001040C1F80C057047E41902000249085CF6
:10ABE000012103F0FCB80000E41902000249085CEE
:10ABF000002103F0F4B80000E41902000649095CE2
:10AC00004FF0A040D0F80405C84010F0010000D07B
:10AC1000012080F001007047E419020010B5002403
:10AC20002046FFF7DBFF641C042CF9D310BD10B5E0
:10AC300000242046FFF7DAFF641C042CF9D310BD72
:10AC400010B50246064B4FF0FF3000215C5C944289
:10AC500001D1084610BD491C0429F7D310BD0000DE
:10AC6000E819020070B50C4E0C004FF00005306082
:10AC70000BD0012000F06AF808B1022004E00020A7
:10AC800000F064F800B10B202070706810B9FEF776
:10AC900069FF0546284670BD601B002010B50020E6
:10ACA00000F0D4F908B1062806D1012000F0CEF951
:10ACB00008B1062800D1002010BD00002DE9F047A2
:10ACC0000D468146FFF7BCFF0446042836D2DFF864
:10ACD00074801B481C4EA8F10C0725B3012D0ED023
:10ACE000022D2BD104EB440030444578002D25D0B3
:10ACF000B968002922D02846BDE8F047084704EB90
:10AD00004401755C0E44717849B10E4A4FF400411C
:10AD1000093A8068FFF76CF808B987F80390B178B2
:10AD200008F80410E2E78068FFF7A6F804EB440196
:10AD3000314418F804008D78A842D7D0BDE8F087D8
:10AD4000EC1902005C1B00204C1E0020042801D2DC
:10AD5000FFF7F8BE002070470146104810B5008884
:10AD6000042907D007290ED00A2915D1BDE81040C3
:10AD700005F06EBE132176DF0CE000280CD0BDE894
:10AD80001040FEF7EDBFA0F57F41FF3904D1044824
:10AD9000FFF728FB0828F0D110BD0000481B002059
:10ADA000541D002070B50023042810D20D4D00EB77
:10ADB0004004012A02D101290CD00022094E00EBE7
:10ADC0004000304461B1012906D0022906D0072392
:10ADD000184670BD0E30C2B22A55F9E74270F7E747
:10ADE0008270F5E74C1E0020044A014600201279CB
:10ADF000D20702D0084600F04DB87047501B002023
:10AE000070B506461E480024C0E90161B00720D590
:10AE10000025012211462846FFF7C4FF6D1C044699
:10AE2000042D02D2002CF4D013E094B940F26662F3
:10AE300004211448FEF71AFF04000AD1FEF704FFAC
:10AE4000040006D10F48104A0021001FFEF794FFAE
:10AE50000446F00712D00120FFF784FE74B90948B8
:10AE60000A4A00210C38FEF787FF040006D1054886
:10AE7000074A01210838FEF77FFF0446204670BDCF
:10AE8000501B0020F819020019B1010029C9010066
:10AE9000379C01002DE9F05F6A4C0546002660787A
:10AEA000B34618B184F801B001F026FD664F4FF4A7
:10AEB0007A694FF4C87A4FF00108182D62D2DFE8A2
:10AEC00005F0AC0C0C31404D62676B746B74BE7D49
:10AED0007D7D7D7DACAFB2B5BEBE0020FFF78EFE9E
:10AEE00000284FF0000008D0FFF778FE022D02D1B5
:10AEF0004FF4E16008E0484606E0FFF777FE022DD8
:10AF000001D1C82000E05046410CC0034FF4FA7252
:10AF1000801841F10001257052000023FEF762FA0B
:10AF200001462AE00020FFF769FE00284FF00000EC
:10AF300004D0FFF753FE4FF44870E5E7FFF756FEE5
:10AF4000DFE70020FFF75AFE00284FF0000002D094
:10AF5000FFF744FECFE7FFF749FED4E70020FFF7F5
:10AF60004DFE00284FF0000002D0FFF737FE01E051
:10AF7000FFF73CFE257041F69A1100223868FEF773
:10AF800037FF064646E00020FFF716FE257008E072
:10AF9000002051E025703DE084F801800120FFF79A
:10AFA0000BFE002240F6CD41E8E784F80180012045
:10AFB000FFF702FE00224FF48041DFE77868FEF7DA
:10AFC0005BFF0646D5F1110000D02EB10220FFF73D
:10AFD00005FE84F802B01DE0012816D980B2C82110
:10AFE0004843C117C90341EA5041C0034FF4FA7204
:10AFF000801841F1000152000023FEF7F3F90146E9
:10B0000000227868FEF7F4FE06460220FFF7EEFD08
:10B0100084F802803046BDE8F09F01F06DFCB9E78E
:10B0200001F06AFCB4E701F067FC04E001F064FCA5
:10B030000020FFF7DBFD0120FFF7D8FDAAE7FFF7AF
:10B04000F6FDA7E7501B0020EC190200012106F0D5
:10B05000B2BA00002DE9F8430546861C00208DF8A1
:10B06000000090460F464FF001096846FEF714FFB6
:10B070001B4C20683860D4E90001401AA16804F232
:10B080001C47081A0EE00121384602F0F2F801F0E0
:10B09000E7FD0146384602F0ECF8D4E90001401A19
:10B0A000A168081A401C8642EDD8B8F1000F03D001
:10B0B000052065F3891002E0062065F39F50A26821
:10B0C0002168114004EB8101C86020683044206091
:10B0D0009DF80000FEF704FF4846BDE8F883000035
:10B0E000F425002030B482680468531C8360A154A6
:10B0F000D0E901128A4202D330BC02F0BABA30BCA5
:10B1000070470000034803C8814201D10120704705
:10B1100000207047F425002000780221FFF7CEBD03
:10B1200005494FF0FF32082841F8202002D3084497
:10B1300080F8482070470000B0210020F0B54FF0A3
:10B14000FF3512B10023082601E008230C260C4C21
:10B1500005E000BF54F823707F1C04D05B1CB34291
:10B16000F8D32846F0BD26185DB286F8305044F872
:10B170002310002AF5D1E11881F84800F1E700001A
:10B18000B02100200249084490F9300070470000C7
:10B19000B021002070B504464FF6FF750A462846D8
:10B1A000AC4208D14FF480742146104604F05EFD95
:10B1B000A04209D070BDFF2CFCD82146104604F0F7
:10B1C00048FD08B1204670BD284670BD70B5084CDA
:10B1D000050009D010342168002907D008682060D4
:10B1E000496828468847F6E70834F4E770BD000050
:10B1F0009C210020054A012120B1012805D1917030
:10B20000FFF7E4BF51700020FAE770479C2100204F
:10B210002DE9F05F26484168F1B3DFF898B00E6879
:10B220008146DBF8004087688078E11B21F07F458C
:10B23000ED1CB0B9DFF880804FF48030C8F84403CB
:10B24000C8F804031120FEF749FA1120FEF751FA5D
:10B250004FF0010AC8F800A02F2003F011FC89F874
:10B2600002A0B54200D23546124BE8193C3320F01B
:10B270007F401860DBF800105A46091B21F07F411F
:10B28000001B20F07F40C91C81420FD91068186054
:10B290002F2003F0F5FB00E004E0BDE8F05F112093
:10B2A000FEF732BABDE8F05F05F0FCB8BDE8F09FEC
:10B2B000F81B0020041501400010014073B58CB04C
:10B2C0000646002000900D9880B100246D4621466E
:10B2D0000DA801F0B0FF30B1009805EB400084806C
:10B2E0000098401C0090641C142CF0D32C2269465A
:10B2F0003046FEF7BBF80EB070BD2DE9F04117885F
:10B300000646B81D14460D46984202D90C20BDE8E9
:10B31000F0813188072206290AD34FF4486C4FF692
:10B32000FF73614501D9994202D17088062801D284
:10B330001046ECE7604501D99842F9D1994203D013
:10B34000984201D08142F3D80520E8552088122187
:10B35000401C80B2208029542088401C80B220806C
:10B360004119308805F0D6FF2188084480B220803A
:10B370004119708805F0CEFF218808442080002004
:10B38000C5E7FEF7EDBC000038B54A7A0F4B62B155
:10B3900000220A725969002906D001228DF8002086
:10B3A000ADF802006846884738BD0A7A62B19B68EA
:10B3B0004C68024619462046FEF71AFD0028F3D0D5
:10B3C000BDE8384005F048BA5B68F1E7AC1E0020E4
:10B3D000F0B585B016460F4604461D4614220B49AB
:10B3E0006846FEF743F80A488DF80870ADF8024049
:10B3F000ADF80A608DF80C50017800222046FFF766
:10B400009DF9684600F0FAF905B0F0BDFC1A02009B
:10B41000A81B002030B5044685B000211B4804F06D
:10B4200018FC00282FD00025204600F0C4FE68B18B
:10B43000112812D086281BD0A0F54051023903D024
:10B440000146204605F010FA294607E005B02946D6
:10B450002046BDE8304001F0E1BB0121204601F06B
:10B46000DDFB05B00021BDE83040084804F025BCF4
:10B47000142207496846FDF7F9FFADF80240684617
:10B4800000F098F9E0E705B030BD0000711B002026
:10B490002C1A02007FB50C4610B1012004B070BD1B
:10B4A0002079002638B141F61D5501281BD002280D
:10B4B00026D00F20F2E70220207102960396E06862
:10B4C0000190694601A804F049FF50B102988188B3
:10B4D000E18000882081BDF80010029804F0BCFFD4
:10B4E000DCE70A20DAE70A4B6A460021A01D04F0D7
:10B4F000F1FE38B1064918398E61CE610A28CDD1E6
:10B500002846CBE702488188019804F0A5FFF5E7BB
:10B51000381C00202DE9F0470025DFF88C803CE046
:10B520006068002100EBC506012032789146FDF7E6
:10B530008AFFD4E9062300EA020701EA030C57EA6E
:10B540000C0728D082438B434846C4E9062303F006
:10B5500059FB32788246914601200021FDF773FFA6
:10B56000D4E9042300EA020401EA03074A465046EC
:10B570000021FDF768FF44404F403C430BD17078F9
:10B58000012801D0012100E00021726881EA0A014E
:10B590000AB1484690476D1CEDB298F80000444649
:10B5A0008542BDD3BDE8F087D81B002010B500212F
:10B5B000024801F079FE80F3100010BD102A00202F
:10B5C0000E4910B50A784C780023A24212D0521CC2
:10B5D000D2B20A70022A00D10B70084A0B780C32E2
:10B5E00052F8232002608868104420F07F40886071
:10B5F000012010BD0360002010BD0000F81B0020DA
:10B6000013460A460021FFF7E3BE00002DE9F84388
:10B61000104D0F4680461E4691466946286801F047
:10B620009EFD040014D01C21FDF739FF012020717C
:10B63000C4F81490380BC4F80080C4E9026069466D
:10B64000286801F0ADFD04F0D9FD0020BDE8F883C5
:10B650000420FBE7C81B020010B503780022072B6B
:10B6600006D2DFE803F005040610202930000A7036
:10B6700010BD01230B7003898B818388CB81C06847
:10B6800088600A7410BD02220A7002898A81828849
:10B69000CA81C2688A60807D062802D000200874B2
:10B6A00010BD0120FBE703220A70C2888A8102894B
:10B6B000CA81C068886010BD04230B70C08888816F
:10B6C000CA818A6010BD0520087010BD70B5064D96
:10B6D0000646002455F8241009B130468847641CFA
:10B6E000042CF7D370BD00007423002030B504464D
:10B6F000006887B00D46806800281FD01821684672
:10B70000FDF7CDFE0195A0680590207910B10128C4
:10B7100010D107E001208DF8000020690290E06858
:10B72000039005E002208DF80000E068000302901D
:10B7300060690490206881686846884707B030BD1A
:10B7400070B586B015460C00064619D0112C17D0DE
:10B75000082C15D014216846FDF7A1FEADF8026053
:10B76000304600F01FFFADF804000D2C0AD0862CE7
:10B770001CD007208DF800000294684600F04CF8B9
:10B7800006B070BD03208DF8000025B12878C007F1
:10B7900001D0012000E002208DF8080000208DF883
:10B7A0000C0041F20110ADF80A00E6E706208DF822
:10B7B0000000E2E710B50446408800F0F3FEA080E8
:10B7C000024801682046BDE810400847781B002069
:10B7D0002DE9F04107460024064E074D05E000BF65
:10B7E00056F8241038468847641CE8788442F7DB12
:10B7F000BDE8F08150210020981B002010B50446C0
:10B80000408800F0CFFEA080024801682046BDE8D5
:10B8100010400847D01A0200014909680847000093
:10B82000241B020070B586B0044614216846FDF75B
:10B8300036FEA0890125A0F54040ADF8040020782F
:10B840002A4E062833D2DFE800F0320303032C48E7
:10B85000A08900F0BDF930B9E08943F6FE71A0F58A
:10B860004040884223D8A07B8DF808002078032828
:10B870000FD000208DF80900A0680390606850B1D7
:10B8800009208DF8000060680490684603F046FEC9
:10B890000DE00120EEE708208DF800008DF8105033
:10B8A000F3E7A08900F094F908B1E08930B170782D
:10B8B000002801D003F062FF06B070BD606820B1BF
:10B8C0000B208DF800007570DFE70A208DF800006E
:10B8D000BDF8040003F0DCFFF5E713208DF800004D
:10B8E0004FF6FF70ADF80400CFE70000881B002082
:10B8F00038B504460E480078A8B1A4F57F40FF385B
:10B900000FD0684604F0ACFB78B10521017001212D
:10B910000171C480684604F0B1FB04F061FC0020B2
:10B9200038BD042038BD022038BD082038BD0000D5
:10B93000401C00200C4808B5007888B1684604F027
:10B940008FFB78B106210170684604F097FB074829
:10B95000017809B10121017304F042FC002008BD07
:10B96000022008BD082008BD401C0020382400200B
:10B97000F0B587B014216846FDF791FD2B4C207877
:10B9800018B16846FFF7A2FE4EE0201D01F06EFCE4
:10B99000B8BB4FF010204169000400694A1C02D175
:10B9A00000EB40000101224800220161A1F5405155
:10B9B000C160204901F0ECFF002820D11F481C2362
:10B9C0008C221D49006801F0B7FB03F097FB0500CE
:10B9D00014D0022D12D000270126062D12D005A862
:10B9E00004F03EFB88B106700C2D18D2DFE805F09C
:10B9F000170F170F17161716171113110B2007B073
:10BA0000F0BD11E026706760BBE70820F7E707711B
:10BA100005E0032100E00221017100E0067105A8A4
:10BA200004F02CFB04F0DCFB0020E8E7401C0020C5
:10BA3000E81C0020D81B020084230020401B0200C9
:10BA400038B5040014D0694604F088FCA0B1BDF8F4
:10BA5000000000EB8001094800EB8100C16849B19A
:10BA6000A17A39B1C168491EC1600020A07238BDF9
:10BA7000052038BD062038BD0A2038BD102400201E
:10BA80001FB501A9684604F025FC04B010BD07B538
:10BA900013460A466946002004F01CFC0EBD07B59B
:10BAA00013460A460021684604F014FC0EBD20B17E
:10BAB00019B1006808600020704705207047000039
:10BAC000F8B50D46040018D0BDB1694604F046FC37
:10BAD000A8B1BDF800000B4900EB800001EB80002D
:10BAE00001210C30666801F0C4FB2E6060680C30E8
:10BAF00068600120A0720020F8BD0520F8BD0A2072
:10BB0000F8BD00001024002018B10323002205F026
:10BB100041BE052070470223002205F03BBE12B152
:10BB2000022305F037BE052070470000084910B514
:10BB30000A69042A0AD0074A096942F82100044820
:10BB40000121103001F095FB002010BD0C2010BD2C
:10BB5000201C00207423002038B5044609480D46F7
:10BB6000007858B164B16946284605F00DFF0028F9
:10BB700003D1BDF800102180658038BD022038BD9A
:10BB8000052038BD401C002010B504460E48007842
:10BB900098B1A4B12188022913D80C4A01EB810085
:10BBA00002EB800260885289C31C934209D805F0D9
:10BBB000DFFE00202080608010BD022010BD052027
:10BBC00010BD042010BD0000401C002010240020E7
:10BBD00043F6FE71A0F54040884201D8012070472D
:10BBE0000020704710B504460078182802D1FEF7EF
:10BBF00081FD207010BD10B504460078182802D1D0
:10BC0000FEF778FD207010BD70B50D460446B0F803
:10BC10009810D0F894000122FEF7EBFA00B10570FD
:10BC200004F13C0204F1940104F1540072DF70BD90
:10BC300070B51346002206461546862902D0112902
:10BC400002D002E0012200E001250D4C73B1A17980
:10BC5000FEF774FD2A4661793046FEF76FFD00223B
:10BC6000A1783046FEF76AFD002203E0A178FEF7D6
:10BC700065FD2A4661783046BDE87040FEF75EBD3E
:10BC8000B01B0020F7B517460E0011D00098002514
:10BC900060B100242146684601F0CDFA18B1A0B287
:10BCA0003946B0476D1C641C142CF3D32846FEBDE6
:10BCB0000020FEBD406804F0F3B9000070B508B183
:10BCC000012070BD194C0025207B08B1257301E0CF
:10BCD00000F0A0F82078082826D2DFE800F025043C
:10BCE000080C10251420BDE8704000F021B8BDE814
:10BCF000704000F07DB8BDE8704000F05FB8BDE86E
:10BD0000704000F03BB86088084900EB800028399B
:10BD100001EB80004068BDE8704003F0CFB965607A
:10BD2000BDE8704003F0D8B90F2070BD3824002062
:10BD30001149F0B48A1C00200346A1F128050C1813
:10BD4000A67A4EB1A37200EB800405EB8404E6688A
:10BD500016B9247C012C0AD0401C80B20228EED3F4
:10BD60000B704B804B60F0BC41F61D50704710804B
:10BD7000F0BC00F03DB80000382400200C48418899
:10BD800001EB8102A0F1280101EB8201CA6852B1E6
:10BD900005210170074802218180016800230122EA
:10BDA000054801F05FBD042202704968F6E7000013
:10BDB00038240020481C0020E81C002038B50A491F
:10BDC000084803240B684268898803EB8101538883
:10BDD0000470DB1C00201B0400909B0B034801F047
:10BDE000B1FE38BD38240020481C0020E81C00208B
:10BDF000074910B54888091D04F000FB18B1BDE8DB
:10BE00001040FFF7DBBFBDE81040FFF7B7BF0000F1
:10BE100038240020F0B51F481F4901250678022468
:10BE20008B88A0F12802082E19D2DFE806F004184A
:10BE3000181B222F2F170189491C018100214180E5
:10BE400080F80C1001EB810312F8233043B100237A
:10BE50004418491C89B2A3720229F3D30570F0BDBE
:10BE60000123F5E742685288D21C1A448A80047084
:10BE7000F0BD46880D6806EB860602EB8602566822
:10BE80000E60556013818C80062100E0072101704F
:10BE9000F0BD000038240020481C002030B5018887
:10BEA0008488224D85B0502924D0522902D05429AB
:10BEB00031D103E0204600F07DFE2CE014221C4925
:10BEC0006846FDF7D3FAADF80240204600F06AFB61
:10BED000ADF8040000F022F9002269792046FEF74F
:10BEE0002DFC002229792046FEF728FC6846FFF742
:10BEF00061FC10E0017B01290DD1817A01290AD171
:10BF00000089A0F52451023905D10121204600F015
:10BF100085FE05F06FFA00220649E878FEF7CCFBB3
:10BF200005B0BDE8304004F0DDBC0000701B00200F
:10BF3000541A02009D9F010010B5044600780028A5
:10BF40000FD1608800F036FE608800F081F900288B
:10BF500007D00449608801220979BDE81040FEF746
:10BF6000EDBB10BD701B002010B5124C00202070DE
:10BF7000FEF7C0FBA070FEF7BDFBE070FEF7BAFB5A
:10BF80002071FEF7B7FB6071A17818290FD0E17816
:10BF900018290CD02179182909D0182807D0012197
:10BFA000601C03F04FFE01202070002010BD032014
:10BFB00010BD0000701B00207CB5044600780828E6
:10BFC0002FD1607A38BB207A4FF6FF7501280DD04B
:10BFD000072802D0082824D11EE0A08800F020FA0B
:10BFE000A8421ED0012100F019FE1AE0A0886A467E
:10BFF000012103F0ABF970B90198007858B1A0881D
:10C0000000F00EFAA8420CD0084901220979FEF787
:10C0100095FB04F067FC04E004480021401C03F099
:10C020004CFEBDE87C4005F0E5B90000701B002027
:10C0300010B504460A4841782046FEF767FB68B110
:10C040000848002101EB410200EB82025288A24223
:10C0500001D1C8B210BD491C1429F3D3FF2010BD73
:10C06000821B0020401F002070B5094D094E00249E
:10C0700004EB440005EB800071784088FEF746FB36
:10C0800020B1641C142CF3D3FF2070BDE0B270BD4E
:10C09000401F0020821B00202DE9F041804602460F
:10C0A00001200021FDF7CFF91A4F05460E467868AA
:10C0B000FDF7E2FE00280CD1174CD4E9062110460A
:10C0C0002A4001EA06031A4305D0A843B143C4E954
:10C0D0000601BDE8F081404602F094FD30B1D4E99C
:10C0E000040128433143C4E9040105E0D4E9041004
:10C0F000A943B043C4E90410D4E9060128433143FD
:10C10000C4E90601A1687868BDE8F0410022FDF7A6
:10C110006FBE0000301B0200D81B00201CB5054A72
:10C12000D2E90212CDE900120022694603F033F988
:10C130001CBD00006C1A020003484FF6FF7181809D
:10C1400001210170002070477C1B00202DE9FC417B
:10C15000804600F027FA002403250127A0F57F413F
:10C160002646FF3908D06A46082103F0EFF818B9CF
:10C170000198841D8688056832462B462146404634
:10C18000B1DF042804D0082804D00B2808D002E02E
:10C19000112000E00020002F00D10B20BDE8FC8121
:10C1A0000027A80701D50125E6E73443F5D0002490
:10C1B00026460325E0E72DE9FC41804600F0F2F930
:10C1C0000646A0F57F40FF380ED001252A466D1C9B
:10C1D0000027ADB26B460821304603F0E1F80400B9
:10C1E00006D0072C25D025E043F20200BDE8FC81F3
:10C1F000019903230A1D0B604046891DB2DF04002C
:10C2000004D00C2C09D0052C09D009E032460821B5
:10C21000104603F03BF904460CE0012700E000243F
:10C220000821304603F01EF900B10324002FCDD1C0
:10C2300000E00C242046D9E704488088A0F57F411F
:10C24000FF3901D004F058BB704700007C1B002070
:10C250000EB502A9019100F0A5F96A46012103F08B
:10C2600075F808B100200EBD019800780EBD0000E1
:10C270002DE9F04107464FF6FF760A48B3DF10B1CB
:10C280000320BDE8F081074C43F20305A41E3246AB
:10C2900061883846AFDFA842F3D16088401C6080D7
:10C2A000F5E700007E1B0020428800EB82020C3282
:10C2B0008A4201D9022070478188A1F57F42FF3A66
:10C2C00003D0008808B100207047012070478842E1
:10C2D00004D20068401C01D0012070470020704744
:10C2E0003EB5027802230C46B3EB520F17D1B0F8DB
:10C2F0000110ADF80010C1788DF802108188ADF8FA
:10C30000041080798DF8060002AA01A92046FDF7E5
:10C3100069FC032202A96846FDF7D3F808B10020A2
:10C320003EBD01203EBD000010B50C46FFF780FE6B
:10C33000FF280CD0074900EB400001EB800041686A
:10C3400021600189A180807AA071002010BD0520A4
:10C3500010BD0000401F002070B5018890B010296A
:10C3600059D1011D28226846FDF780F89DF8040088
:10C370004FF6FF76032134466D46B1EB500F2AD0BD
:10C3800003F03AF99DF8040040080ED001280CD0C3
:10C39000022820D118E00C99281D1131FDF7BDFBB2
:10C3A00018B100BFBDF8284015E00BAA0AA9072064
:10C3B00003F0F6F80028EED10DE00C99281D491C79
:10C3C000FFF78EFF0028EDD10BAA0AA9072003F082
:10C3D000E7F80028F1D1BDF80000291D00F056FE55
:10C3E000B44218D0BDF80000214600F0C5F8BDF8F1
:10C3F0000000ADF82A000020ADF82C40074E8DF863
:10C4000028000AAD044600BF56F824102846884785
:10C41000641C022CF8D310B070BD0000801A02001A
:10C42000094A002101EB410332F82330834205D150
:10C4300001EB410002EB800040887047491C142941
:10C44000F0D34FF6FF707047401F00203EB50C46FA
:10C45000054603F0D1F80BE0BDF80000A04207D07C
:10C460002846029900F02EF810B1BDF800003EBD3C
:10C4700001AA6946072003F093F80028ECD14FF693
:10C48000FF703EBD10B50D4C18200D4A60700020A5
:10C490004FF6FF7100EB400302EB8303401C598011
:10C4A0001428F7D3FEF726F96070182803D001206E
:10C4B0002070002010BD032010BD0000821B002052
:10C4C000401F00202DE9F0410C46054600F1110700
:10C4D00001F111061022491C401CFCF7F2FF48B97B
:10C4E000681C00F0F9F928B1601C00F0F5F908B1FA
:10C4F000012400E0002431463846FDF70EFB3B786E
:10C500000222B2EB530F0CD00321B1EB530F08D032
:10C510003378B2EB530F04D0B1EB530F01D00121AC
:10C5200000E00021084201D18C4302D00120BDE887
:10C53000F0810020FBE7018811B9421892780AB116
:10C5400001207047491C0829F7D30020704710B517
:10C550000C460346FFF7EFFF00280AD01888218811
:10C56000884205D10822A11C981CFCF7AAFF08B13B
:10C57000002010BD012010BD03F0DEB970B50446E7
:10C58000FFF74EFF0546204602F0E3FE4FF6FF712F
:10C5900004468D4203D014B9284603F0CDF9204655
:10C5A00070BD000010B5FFF743FDFF2805D004491A
:10C5B00000EB400031F8200010BD4FF6FF7010BDB9
:10C5C000401F00203EB5044603F016F80EE0019926
:10C5D00020464631FFF7BBFF28B9019920462A3192
:10C5E000FFF7B5FF10B1BDF808003EBD6A4602A9CD
:10C5F000072002F0D5FF0028E9D14FF6FF703EBDBD
:10C6000010B50A4941600A4800F030FE58B902F0FE
:10C6100077F907491C238C22087404488C39001FC1
:10C62000006800F089FD002010BD0000CC1B020056
:10C63000D42400202DE9F0412D4F002518B17D6054
:10C640000120BDE8F0810879012258B1294E012866
:10C650000CD0274C4FF002080834022821D00328C0
:10C6600042D128E00A7102F037FD3BE05FF00000A4
:10C6700000EB800116F82110022908D0401C80B27E
:10C680000228F5D33A707D6041F61D50D9E700EBE2
:10C69000800006F8205006EB8000406802F00EFD96
:10C6A00020E00D71A4F804800023012212482168C3
:10C6B00001F0D8F816E00D71206802F0FFFC0D497A
:10C6C00023682831498801EB810206EB8201D1F809
:10C6D00004C0C4F800C04B60A3880B81A4F8048098
:10C6E00006F822500028ACD07D600E20A9E700009B
:10C6F000401C002010240020E81C002001460348B4
:10C7000002888A4200D0002070470000981E002056
:10C710002DE9FC5F0E008346DDE90C47C6F1000001
:10C7200098469246814600D40846012503E000BFA2
:10C7300090FBFAF06D1C5045FADAA84500D9454641
:10C7400024B1002E01DB780700D5641EB80702D59E
:10C75000B8F1000F0AD0F80708D13CB1A54205D2C4
:10C7600020215846641EFEF7BDFCF6E7002E02DAD3
:10C770004E462D2102E0780703D52B215846FEF7BF
:10C78000B1FC07F0030002280BD1B8F1000F08D16B
:10C790003CB1A54205D230215846641EFEF7A2FCEA
:10C7A000F6E7CDE90047434652463146584604F085
:10C7B000C7FDBDE8FC9F000070B50D46044600684B
:10C7C0004FF4887102F021F94FF49071206802F063
:10C7D0001CF94FF49271206802F017F94FF4A2711E
:10C7E000206802F012F920681249C0F8041320688A
:10C7F0006907000B40B2090E002806DA00F00F00AE
:10C8000000F1E02080F8141D03E000F1E02080F842
:10C81000001420680121000B40B200F01F0291407B
:10C820004009800000F1E020C0F88012C0F800113B
:10C8300070BD00001003020002460020126893073A
:10C8400002D0530702D47047500714D502F00300FA
:10C85000012802D002280CD105E0C2F383100B6836
:10C86000801C184404E00223086803EB9252104431
:10C87000086001207047086800EB9253C2F38910EA
:10C88000401CEEE70248007A002800D001207047E3
:10C89000D4240020F0B58488A518944200D82246FC
:10C8A000A41AC288D6189A4200D81346D21A4B88C6
:10C8B0000788BB420CD34088834209D88888A042AD
:10C8C00006D3A84204D8C888904201D3B04201D907
:10C8D0000020F0BD0120F0BD0021425C0AB1012022
:10C8E0007047491C1029F8D300207047800701D0F9
:10C8F00000207047012070470A4810B5807860B169
:10C90000002401E0022C06D02046FEF767F9641CE3
:10C91000042CF7D310BD0324F6E7BDE81040FEF762
:10C920007DB90000501B002003480179C90702D0DF
:10C930000078FEF7AFBA7047501B00201721018026
:10C940004180002101714171704700002DE9FE4FC7
:10C950002B4D984691460F00824601D000260DE0EF
:10C96000684600F0BFFB6A460021504602F05DFCBD
:10C970002878009E10B99DF8090098B14A463146C2
:10C98000504604F0D5F90446014600225046FFF710
:10C990004FF90D2C32D008DC84B3082C2ED00B2C90
:10C9A0000BD12BE00520BDE8FE8F112C10D0862C7A
:10C9B0001AD0A4F54050023820D00325B8F1000F5A
:10C9C00004D0324621465046FEF7BAFE2846EAE732
:10C9D0003A4629795046FDF7B1FE4A46E978504675
:10C9E000FDF7ACFE0025E9E73A4629795046FDF708
:10C9F000A5FE4A46E9785046FDF7A0FE2546DDE74C
:10CA0000B01B00202DE9F041204F0E46154604468C
:10CA10003978FDF77BFE002835D0204602F0FCFB7C
:10CA200050B32046FFF7BEFD80462046B978FDF79B
:10CA30006DFE08B1012700E00227204602F094FEB7
:10CA40000028404602D0FFF799FD0DE0A8F57F4190
:10CA5000FF3909D0072102F005FD010004D00529A6
:10CA600002D0204603F014FF2B46324639462046BA
:10CA7000BDE8F041FEF7ACBC2A4631462046BDE891
:10CA8000F041FEF7BDBDBDE8F0810000A81B00200D
:10CA900070B5094D0646E978FDF738FE0446297958
:10CAA0003046FDF733FE014622463046BDE8704071
:10CAB0000123FFF74BBF0000B01B00202DE9F0471A
:10CAC000394E002780463D46DFF8E090D6F804A0B6
:10CAD00057E003D00446D0F81C8035E099F80020D8
:10CAE00002EB4201521CD2B289F8002009EBC101CD
:10CAF00099F80230091D9A4201D189F8005048681E
:10CB00000A780446012A12D0022A02D0032A3BD115
:10CB100008E004F0B1FA00B10127257434E005748F
:10CB2000C06900E070680028F9D170602CE0207CBA
:10CB300050BB88686060C868A0600869E0604869A8
:10CB4000A061F07800B165606268B168184B501A56
:10CB500020F07F40984202D2A168084406E0881A7B
:10CB6000A16820F07F40814202D9081A206000E0CD
:10CB7000256065600120A56020742046E56104F011
:10CB80005DFAB8F10000A4D199F8001099F80100FD
:10CB90008142A3D117B97168514502D00120BDE887
:10CBA000F0870020FBE70000F81B00205022002047
:10CBB000FFFF7F0030B585B005460024142168468C
:10CBC000FCF76DFCA5F57F40ADF80250FF3815D09D
:10CBD0002846FFF7BBFA98B10B2815D0112811D0C1
:10CBE000A0F54051023903D00146284603F03CFE2F
:10CBF00009482246C1782846FDF7A0FD05B030BDA2
:10CC00000E2002E00124F3E70F208DF800006846B3
:10CC1000FEF7D0FDECE70000701B00200A46024939
:10CC20008978FDF78BBD0000701B0020F8B5054624
:10CC300000780C46002620420FD100208DF800001D
:10CC40006846FDF729F92878204202D12043287050
:10CC500001269DF80000FDF743F93046F8BD0000BD
:10CC60002DE9FF410026234800F0FDFA2148001F6E
:10CC7000074600F0F8FA204C60680090A56800E0D4
:10CC800000986946284004EB80000C30FFF7D4FD83
:10CC90000028F5D101AA009901EA050304EB8303FA
:10CCA000491CDB6842F82030401C00910228F2D376
:10CCB000019800F0030001280BD0022810D1019840
:10CCC000032101EB90500099BDF80A6001EB900040
:10CCD00005E00198BDF80A60C0F383100844009095
:10CCE000384600F0BDFA08B10098606004B03046E4
:10CCF000BDE8F0810C2A0020F4250020ACB04FF4F0
:10CD00000041002001F0ECFA08B1FDF729F801F02C
:10CD100057F9FDF743F808B1FDF722F85E49032003
:10CD2000FEF76EF808B1FDF71BF869460020FDF725
:10CD300099FF08B1FDF714F89DF8000002287CD097
:10CD40005FF0000501F0EAFB08B1FDF709F801F01A
:10CD50007DFD08B1FDF704F8002469460120009428
:10CD600001F006FC08B1FCF7FBFF684601F080FC0F
:10CD700008B1FCF7F5FF9DF8080048A120F00F006E
:10CD8000401C20F0F00010308DF808000F2202A89F
:10CD90007CDF08B1FCF7E4FF00945020ADF8000000
:10CDA000A0200194ADF80200ADF804404FF4C87023
:10CDB000ADF8060068467ADF08B1FCF7D1FF002124
:10CDC0003A4800F0E6FA08B1FCF7CAFFAC21684621
:10CDD000FCF765FB02208DF8000001208DF80200B1
:10CDE0000621ADF810008DF87C008DF803104FF48B
:10CDF00096702F492290059144F2506023902D485F
:10CE000029902A4869461C30FDF722FA08B1FCF740
:10CE1000A7FF264801211C30FDF717FA264800908D
:10CE200022486946103000F046FB08B1FCF798FF35
:10CE30001C216846FCF733FB00E02AE04FF4203069
:10CE4000CDE900404FF4702002901C480590032665
:10CE50001B488DF80C600690ADF80E408DF8104020
:10CE60006846FDF7E5FB08B1FCF77AFF02F072FDBA
:10CE7000144815A1008806EB004001F0BFF92846D0
:10CE8000FCF78CFE01F0AAF80028FBD101F05AFB58
:10CE9000F8E7012556E7000059AD01004E6F7264B6
:10CEA00069635F54656D706C61746500381D0020A6
:10CEB0004A1B00207DEE010059E50100C9EE01008A
:10CEC00083B30100281D002054656D706C6174658A
:10CED000206578616D706C6520737461727465642F
:10CEE0002E00000070B5144682880E460546208844
:10CEF000111D0144921C994201D8FE2A01D90C202F
:10CF000070BD521C32542088FF21401C80B220800A
:10CF100031542088401C80B220808119288804F078
:10CF2000F9F92188084480B22080AA8842B1A96812
:10CF300041B13044FCF79AFA2088A988084420803F
:10CF4000002070BD072070BD2DE9F047C78804465A
:10CF5000181D16468946B0FBF7F1B0FBF7F207FB48
:10CF600012009A193A44D21CB2FBF7F2DDF820A065
:10CF700001E02468491E0029FBD13D1A8846B542CC
:10CF800016D818E0BAF1000F05D0211809EB0800F7
:10CF90002A46091D04E0204409EB08012A46001D29
:10CFA000FCF764FA00202468761BA844B74201D934
:10CFB000354600E03D46002EE4D1BDE8F087000094
:10CFC00030B5024659B101F0B7F90021074C09E02C
:10CFD00004EB810315685B88AB4202D1116000202D
:10CFE00030BD491C8142F3D3052030BDFC1C00201C
:10CFF000F8B50F46017814460546012901D1687835
:10D0000030B12088821C9A422DD8012902D006E036
:10D010000720F8BD69780144891C994223D8181A61
:10D02000801E86B2ADF800602188B81C08446946AD
:10D030007DDF0028EDD12878022805D1BDF8001049
:10D04000B14201D809210AE00821012805D16878F8
:10D05000B04202D8ADF8000001E0ADF80060BDF8C4
:10D060000000FE2801D90C20F8BD2288401CB854CD
:10D070002088401C80B2208039542088401C2080A9
:10D08000BDF80010084420800020F8BD70B50546AA
:10D090000C004FF0FF0020D04FF6FF76B5421CD0B9
:10D0A0000E48012241782846FDF748FB2846FEF746
:10D0B000BFFFFF2803D1FEF7D7FFFF280DD0084B95
:10D0C00000EB400203EB82014D8023F822602268CE
:10D0D0004A60A2880A81A2798A7270BD821B0020F0
:10D0E000401F0020034A00219268C0E900218160AE
:10D0F00070470000B01B002070B54FF6FF750E465C
:10D10000A84201D1002000E0401C84B208E0214682
:10D11000304602F0C6FD08B1204670BD641CA4B2C2
:10D12000FF2CF4D9284670BD10B5FCF7BEF808B145
:10D13000002010BD112010BD10B531B1B2FBF3F4C9
:10D1400003FB14241CB1092010BD0E2010BD01608A
:10D150000021416081608281C381084610BD70B5A5
:10D160000C460546FCF756F8002802D021882868AE
:10D17000084470BD10B50A8849888A4203D1FCF77B
:10D180008BF8012010BD002010BD70B50C4605467F
:10D19000FCF765F8002802D061882868084470BD53
:10D1A00010B50A8849888A4203D1FCF74FF801205C
:10D1B00010BD002010BD01F01F0301229A40D24390
:10D1C000490900EB8100114600F059B80A4601F008
:10D1D0001F030121994010B552090C4600EB820053
:10D1E00000F05DF8204000D0012010BD2DE9F04195
:10D1F00080460D460024481E012101EB501716E021
:10D2000058F82400C04390FAA0F0B0FA80F020282B
:10D210000CD200EB4416AE4208D231464046FFF72E
:10D22000D5FF0028ECD13046BDE8F081641CA74250
:10D23000E6D82846F8E74A0950F8220001F01F0214
:10D2400001219140084000D00120704701F01F03E8
:10D2500001229A40490900EB8100114600F029B8EB
:10D26000002100F017B8012100F023B8012100F0DF
:10D2700016B808B56A46FCF764F8009808BD08B50A
:10D280006A46FCF744F8009808BD08B56A46FCF702
:10D2900058F808BD08B56A46FCF739F808BD08B566
:10D2A0006A46FCF727F808BD08B56A46FCF716F889
:10D2B00008BD08B56A46FCF71DF8009808BD08B51A
:10D2C0006A46FCF74BF8009808BD38B504460025BF
:10D2D0008DF800506846FCF7DFFD21686268086839
:10D2E00090420ED9401E08600178A38AE26801FBD3
:10D2F0000325227A2168101AC0B20A79824200D22C
:10D3000008719DF80000FCF7EBFD284638BD38B5E4
:10D31000054600208DF800000C466846FCF7BCFD71
:10D32000E868A98A201AB0FBF1F12A681068431C4A
:10D33000136001709DF80000FCF7D2FD38BD10B5F8
:10D3400030B1017A42680368891AC9B21A6006E0EE
:10D350000E2010BD03681A68541C1C601170491E11
:10D36000C9B2F7D2006800210171084610BDC20899
:10D3700000F007030120895C98400840704710B511
:10D38000C20800F00703885C01249C4020438854B5
:10D3900010BD10B560B1C160172120F8021B20F844
:10D3A000021B1B2100F8021BFFF7C8FA002010BD6A
:10D3B0000E2010BD7CB50C468188002933D102882F
:10D3C0000025102A06D0112A09D03A2A0BD0552A56
:10D3D0002ED129E00146204601F084FD28E0A01D61
:10D3E000FFF7ACFA24E02246408934F8063F834236
:10D3F00000D818466080172800D217206080D068B7
:10D4000078B1607968B1174BD3E90003CDE9000327
:10D41000ADF802106088ADF80400D3686946104684
:10D420009847657125717CBD0146204601F09CFD41
:10D43000A07A0028F7D02846E188A5DF012670B140
:10D440001128F0D001F0D2FA0246074807A100885F
:10D4500002B006EB0040BDE8704000F0D3BEA572FC
:10D46000E6727CBD881A0200FC1C002073645F62B7
:10D470006C655F67617474635F65786368616E672C
:10D48000655F6D74755F72657175657374282920A9
:10D4900072657475726E65642025732E000000003D
:10D4A00020B10278DE2A03D0082070470E20704792
:10D4B00041800020704760B159B10278DE2A0AD05D
:10D4C00009684160DE2101704FF6FF714180002044
:10D4D00070470E207047082070477FB50546002929
:10D4E0004DD0002D4BD008780C46DE2847D1A888B7
:10D4F0006188884202D1204603F0CCFF28880128A9
:10D5000025D002283BD011283AD0512837D135F800
:10D51000040F6188884232D1A978A81C02292ED133
:10D52000017A042903D0062901D0052927D1002139
:10D53000009102228DF8002001914FF4C0720291F7
:10D540000391ADF80420007A05280FD010E0297A65
:10D550002046012913D1A988428891420FD1012187
:10D56000017204B0BDE8704003F094BFADF8041040
:10D5700028886946B0DF002801D0616888477FBDF0
:10D58000A88861888842FAD14FF6FF7060807FBD1D
:10D5900000F180400068002800D00120704708B5E5
:10D5A00000F18040002101600068009008BD00008B
:10D5B00070B50B4C207808B185250FE00020A060E5
:10D5C00060602061E060074801F03CFA054601F028
:10D5D00097F908B901F020FA01202070284670BDA3
:10D5E0009C210020F5B1010038B500258DF80050D0
:10D5F0006846FCF751FC074CE068401EE060E068BC
:10D6000010B901F02FFAA5709DF80000FCF768FC36
:10D6100038BD00009C21002070B5064604780C48F7
:10D6200088B0154640F82420094A0869121D42F8BE
:10D63000240020226846FBF719FF04940DB1054A27
:10D6400000E000226946301D01F034FB08B070BDD7
:10D65000C81B0020F11102000FB408B5039900297E
:10D6600004D004AA00926A4600F00FF801B05DF8F9
:10D6700014FB10B582680446002A05D0D4E90403DF
:10D68000216898470020A06010BD2DE9FC47914615
:10D690000C00804676D014F8011B39B125290ED034
:10D6A0004046FDF71FFD20780028F4D198F80C00C3
:10D6B000002867D04046BDE8FC47FFF7DABF0020EE
:10D6C000012221782B291BD02D2902D0302908D105
:10D6D00002E040F0010001E040F00200641C002A7A
:10D6E000EFD100252A290ED02178A1F130020A2A93
:10D6F00011D205EB850201EB4205641C303DF1E7D8
:10D7000040F00400EAE7D9F800100B1DC9F800301A
:10D710000968641C0D44217800232E290BD114F8CC
:10D72000011FA1F130020A2A05D203EB830201EBAB
:10D730004203303BF3E76C290DD068290BD06929EF
:10D7400021D00BDC252918D0582931D063290ED0DF
:10D75000642915D117E014F8011FECE7702969D08E
:10D76000732932D075291BD0782909D120E0D9F846
:10D770000000011DC9F8001001784046FDF7B2FC19
:10D78000641C90E76CE0D9F800100A1DC9F800206D
:10D790000968CDE900500A224046FEF7B9FFEFE7DD
:10D7A000D9F800100A1DC9F8002009680A2206E00D
:10D7B000D9F800100A1DC9F8002009681022CDE927
:10D7C0000050404603F0BCFDDAE7D9F8001000270E
:10D7D0000A1DC9F800200E68C00705D112E04046B6
:10D7E000761C7F1CFDF77EFC31780029F7D104E020
:10D7F000202140466D1EFDF775FCBD42C0D9002DAD
:10D80000F6D1BDE74EB13046FBF754FE074604E0C3
:10D81000202140466D1EFDF765FCBD4206D9002D56
:10D82000F6D103E04046761CFDF75CFC3178002918
:10D83000F8D1A5E7D9F80000011DC9F80010056866
:10D8400030214046FDF74EFC78214046FDF74AFC6A
:10D8500008200021CDE90001034610222946B0E747
:10D86000BDE8FC872DE9F84F2B4E04009A4630881E
:10D870004FF001031546894603EB004024D0216890
:10D8800000292BD0002D32D0626849464FF0100796
:10D890001268A2F1010C1CEA090F11D198466A43E3
:10D8A0002046FCF753F900282AD0206853462A4620
:10D8B000066901B049462046B446BDE8F04F6047CE
:10D8C000164B17A2009721E00E210091134B1EA2C8
:10D8D0001FA100F0A6FC0E20BDE8F88F08210091E2
:10D8E0000E4B26A21AA100F09CFC0820F4E70921A7
:10D8F00000910A4B24A216A100F093FC0920EBE74B
:10D9000000973188054B214A08EB014010A100F037
:10D9100088FC1020E0E70000181D0020B31B020067
:10D92000616464725F69735F706167655F616C6990
:10D93000676E656428705F66732C20706167655F31
:10D940006164647229000000705F6673000000006B
:10D95000257320636865636B206661696C6564206C
:10D96000696E202573282920776974682076616C98
:10D97000756520307825782E00000000705F667392
:10D980002D3E705F617069006C656E00B01E020014
:10D9900038B503000F484FF001054FF00E04008822
:10D9A00005EB004009D061B119600C6801B0A446D4
:10D9B000BDE83040114618466047074B07A2009467
:10D9C00002E0054B07A2009408A100F02AFC0E20FB
:10D9D00038BD0000181D0020681B0200705F6673D0
:10D9E00000000000705F6170690000002573206313
:10D9F0006865636B206661696C656420696E2025CB
:10DA000073282920776974682076616C75652030E9
:10DA10007825782E000000002DE9F04128B101683A
:10DA200019B1C969BDE8F04108470D4D0D48002402
:10DA3000461B14270DE000BF04EB840005EB8000BB
:10DA4000016829B1C969884710B10120BDE8F0819A
:10DA5000641CB6FBF7F0A042EED80020F6E7000009
:10DA6000E81C0020FC1C0020044801214174007ABD
:10DA700008B100207047012070470000D424002026
:10DA8000012801D0032808D10449002201284A7442
:10DA900000D00020087402F053BB7047D42400204B
:10DAA00070B50246022801D0032A45D1234C207AC2
:10DAB000002841D0012833D0022831D1204800234A
:10DAC000022A006802D0032A2AD11BE0E360017910
:10DAD00011B1012924D10DE0D0E90565711B4FF486
:10DAE0008056B14200D33146294481614569A9423B
:10DAF0000ED015E00169491C0161426991420FD1C4
:10DB0000237213E0E168491CE160082908D9E36049
:10DB10002372022A0AD00D21FDF7E8FD02F0B6FAC1
:10DB2000607C28B1BDE8704000F0F0BE0021F3E752
:10DB3000BDE8704002F004BB70BD0000D42400209A
:10DB4000641C00202DE9F84F3A4D04008B462888CC
:10DB50004FF00106DDF828A0984691464FF00E01DF
:10DB600006EB00401AD0B9F1000F1BD02168002944
:10DB700020D00921B8F1000F25D062685368B8FBA6
:10DB8000F3F703FB1782002A21D02B4B2BA2009125
:10DB900035A100F046FB0920BDE8F88F264B3DA2D9
:10DBA000009102E0244B3DA200912FA100F039FB2F
:10DBB0000E20F1E7082100911F4B3AA22AA100F0A4
:10DBC00030FB0820E8E71C4B39A20091E0E75846FB
:10DBD000FBF7B6FF102798B14846FBF7B1FFB0B18D
:10DBE000424659462046FBF7B1FFB8B1CDF800A038
:10DBF000206843464A46C56859462046A847CBE7B1
:10DC0000009728880C4B06EB00402AA20CE00097F6
:10DC10002888094B06EB00402CA205E000972888D5
:10DC2000054B06EB004032A20FA100F0FAFA1020DB
:10DC3000B2E70000181D0020A01B020021286C651F
:10DC40006E202520705F66732D3E705F666C617379
:10DC5000685F696E666F2D3E70726F6772616D5F8F
:10DC6000756E697429000000257320636865636B15
:10DC7000206661696C656420696E202573282920FF
:10DC8000776974682076616C756520307825782E08
:10DC900000000000705F667300000000705F737228
:10DCA00063000000705F66732D3E705F61706900F5
:10DCB0006C656E00616464725F69735F616C696753
:10DCC0006E6564333228646573742900616464721C
:10DCD0005F69735F616C69676E65643332282875AC
:10DCE000696E7433325F7429705F73726329000048
:10DCF000616464725F69735F77697468696E5F629B
:10DD00006F756E647328705F66732C20646573741E
:10DD10002C206C656E29000070B541EA4201DDE9F6
:10DD200004564FF0A04441EA830141EA052104EB87
:10DD3000800041EA0641C0F8001770BD70B541EAA5
:10DD40004201DDE904564FF0A04441EA830141EA73
:10DD5000052104EB800041EA0641C0F8001770BDC0
:10DD600070B541EA4201DDE904564FF0A04441EAB2
:10DD7000830141EA052104EB800041EA0641C0F835
:10DD8000001770BD1CB5002100910B4601220191C6
:10DD9000FFF7E6FF1CBD1CB500220B4600921146A2
:10DDA0000192FFF7DDFF1CBD1CB5002100910B4661
:10DDB000012201911146FFF7D3FF1CBD4FF0A04295
:10DDC00002EB8000D0F8002722F44032C0F8002790
:10DDD000D0F8002742EA0141C0F80017704701223D
:10DDE0004FF0A043824011B1C3F808257047C3F833
:10DDF0000C25704718B5084B6C4601441B6800930E
:10DE000006E000BF54F82030D3F81035401C08C29B
:10DE10008142F7D818BD0000281B0200034908B54D
:10DE20000844002101600068009008BD00600040C7
:10DE300002494058012800D000207047006000408F
:10DE400030B5124B01460020D3F81044224609E0B9
:10DE5000157A854205D1401C0A28F7DB4FF0FF30C8
:10DE600030BD5268002AF3D1421CF9D00872D3F8B1
:10DE700010242AB152684A60D3F81024516030BD92
:10DE80000022C3F810144A6030BD0000F4250020C1
:10DE9000F0B595B01C4615460F4608461A9E00F090
:10DEA0001BFB182109A8FBF7FAFA0E96CDE90954D5
:10DEB0000023082203A9384600F023FB05980690AA
:10DEC000BDF81000ADF81C00BDF81200ADF81E0042
:10DED00000208DF821000398082600F00300012897
:10DEE00002D0022818D032E003983346850AC0F3E6
:10DEF000C2008DF8200003980FA9C0F38314A2007C
:10DF0000384600F0FEFA09A8009006AB22460FA999
:10DF1000284600F03DFA1AE00398840DC0F3C200D1
:10DF20008DF82000082C01D2254600E00825334654
:10DF30002A460FA9384600F0E4FA2E44641B09ABC8
:10DF400006AA29460FA800F075F9002CEAD1384638
:10DF500000F0C8FA15B0F0BD7047012003F020B9F9
:10DF600010B5044800F032FFBDE81040002003F077
:10DF700017B900007C1C002008B5034A009240231A
:10DF8000024AFFF785FF08BDB9080200F42400200B
:10DF90000A4A012902EBC00007D0022907D0032951
:10DFA00007D0042907D000207047022070470420C2
:10DFB000704700797047407970470000A42502003F
:10DFC00010B5FFF7CAFF04210348FFF739FF0249E4
:10DFD0000120487210BD0000841C00202DE9F04F84
:10DFE0008DB0FDF78FF818B100200DB0BDE8F08FAF
:10DFF0007A4C4FF0000BC4F818B4BFF34F8F606831
:10E000000290A568D846284004EB800008E021680B
:10E010000298814201D86160E6E7284004EB800065
:10E020000C3002A9FEF708FC0028F0D105AA0299DD
:10E0300001EA050304EB8303491CDB6842F8203046
:10E04000401C02910228F2D3059800F00300022838
:10E0500002D001284ED0A9E005985022810D8946B2
:10E06000B2EB905F00D850210E4666F39F500590AA
:10E0700008315B4800F0E7F9070079D000F02CFA8E
:10E080004346082205A9384600F041FA029908F1F2
:10E09000080A2940681A8000001D864223D94F4D86
:10E0A0000C3530B1C2B204EB8101301A90460C310C
:10E0B00004E02946F2B2002590462846C6B25346EF
:10E0C000384600F024FA0AEB08032DB132462946FF
:10E0D0004FEA070000F01BFA029909F1030001EB77
:10E0E000900002903BE004EB8101534632463846F3
:10E0F0000C31EFE70598C0F38310062800D3062003
:10E10000059960F38911C1F38310801C059181008A
:10E11000334800F098F9070048D000F0DDF9434695
:10E12000082205A9384600F0F2F908F1080800268F
:10E130000FE00298434600EA0501401C04EB810110
:10E140000290042238460C3100F0E1F908F104088D
:10E15000761C0598C0F38310B042EAD847B1D4F8D2
:10E160001054D4F8180468B1384600F0BBF92FE019
:10E170001CE0687A012804D12A68284639461268CA
:10E1800090476D68002DF4D1384600F0ABF98DF85A
:10E1900000B06846FBF780FED4F8180408B902986E
:10E1A00060609DF80000FBF79BFE11E0D4F810447E
:10E1B00004E021682046896888476468002CF8D10B
:10E1C00008480221008801EB004007A100F016F882
:10E1D000FCF798FF80F0010007E70000F42500201D
:10E1E0001C260200281D00204261636B656E64736B
:10E1F00020666C75736865640000000000231A4691
:10E2000002F096BE08B5012300926A4602F090FE25
:10E2100008BD1CB5CDE9002302236A4602F088FE42
:10E220001CBD3EB5069C8DE81C0003236A4602F027
:10E230007FFE3EBD2DE9F0470E4680461C469246C5
:10E2400008293ED894F80C900020207319461046F7
:10E2500001F0BAFE0025B54206D218F805201AA131
:10E260002046FFF7F9F903E019A12046FFF7F4F97A
:10E270006D1C082DEFD317A12046FFF7EDF90025FF
:10E28000B54210D218F80570FBF7ECF80068C05DD5
:10E2900010F03E0F01D03A4600E02E220EA120469B
:10E2A000FFF7DAF903E00DA12046FFF7D5F96D1C61
:10E2B000082DE5D301222146504601F067FE84F87F
:10E2C0000C90BDE8F0870000202530327800000077
:10E2D000202020007C0000002563000020000000BA
:10E2E000104810B5FF218160002101604160C0F835
:10E2F0001814C0F8141480F820140B4800F0F0F83B
:10E3000000280DD109480A490A4B401AC1080020CB
:10E3100003E000BF23F82000401C8842FAD300200D
:10E3200010BD0000F42500201C2602001C2602005F
:10E33000A4250200FC1C002002480349401AC00822
:10E34000704700001C260200A425020013B5684691
:10E35000FEF736FE08B100201CBD0248009950F8B7
:10E3600031001CBDA425020070B508480125D0F875
:10E37000104480F8205405E0657221682046496801
:10E3800088476468002CF7D170BD0000F425002098
:10E390002DE9FF4781460C9D00200C462F7B2873FA
:10E3A000984616462946184601F00EFE072E42D220
:10E3B000DFE806F004090F161F2A360049462846F2
:10E3C000FFF74AF937E0494628462268FFF744F943
:10E3D00031E0D4E9002349462846FFF73DF92AE019
:10E3E000A0680090D4E9002349462846FFF734F995
:10E3F00021E0D4E90201CDE90001D4E90023494636
:10E400002846FFF729F916E004F1080007C88DE84F
:10E410000700D4E9002349462846FFF71DF90AE022
:10E4200004F108000FC88DE80F00D4E90023494625
:10E430002846FFF711F900222946404601F0A6FDC3
:10E440002F73BDE8FF872DE9F041858A80462D1F97
:10E450004819C01CB0FBF5F0C6B24046FEF735FFC8
:10E46000041E19D00020207101206071E580002772
:10E470002546761EC4F800800BE04046FEF725FFD7
:10E4800060B16179491C6171286005467F1CC0F844
:10E490000080B742F1D32046BDE8F081204600F06D
:10E4A00002F80020F8E72DE9F041457901466B1E9E
:10E4B000002201E00968521C9A42FBD30F68014612
:10E4C000002605E038460C68FEF721FF2146761C41
:10E4D000AE42F7D3BDE8F0810121001DFEF7C9BEB1
:10E4E000FEF72DBF10B504460121001DFEF7E7FE23
:10E4F00010F0FF0F04D12046BDE81040FFF7D3BF56
:10E5000010BD38B501240094FEF71EFD38BD38B5A6
:10E5100000240094FEF718FD38BD0000064910B530
:10E5200000204870091D0860BFF35F8F034904484D
:10E5300000F018FA002010BD6C1C0020101C020016
:10E54000E824002010B500F0DBF908B141DF10BD70
:10E5500020BF40BF20BF10BDFBF702BC20B1034964
:10E5600009680160002070470E207047FC1D020002
:10E57000FEB502460E460846FFF7F0FF002869D1B7
:10E58000002500950195012406208DF80020ADF8A6
:10E59000040002958DF8024069462020326869DF48
:10E5A0002D4F48B100F022FA3988024604EB0143AE
:10E5B0002A491846FFF726FE0095019502958DF829
:10E5C000014069464020326869DF48B100F00EFA28
:10E5D0003988024604EB014321491846FFF712FE31
:10E5E0000095019502958DF800506946012032682A
:10E5F00069DF40B100F0FAF902463888194904EBA6
:10E600000040FFF7FFFD4FF4B060009001950295C8
:10E610006946A120326869DF40B100F0E7F902469F
:10E620003888114904EB0040FFF7ECFD0095019597
:10E6300002958DF800406946A020326869DF40B13C
:10E6400000F0D4F902463888084904EB0040FFF78F
:10E65000D9FD0020FEBD0000301D0020482402002E
:10E6600090240200A8230200F42302005423020095
:10E670002DE9F0410446D0F8008060DF2168194D93
:10E68000074641451CD92888022606EB004016A102
:10E69000FFF7B4FD2888424606EB00401EA1236820
:10E6A000FFF7B7FDF006D0F80C012168800200F1F9
:10E6B0000050421A288825A106EB0040FFF7A2FD72
:10E6C000012467B1384600F091F9024628882AA152
:10E6D00004EB0040FFF796FD3846BDE8F0812E4878
:10E6E0000470F9E7301D0020496E73756666696332
:10E6F00069656E742052414D20616C6C6F6361746A
:10E70000656420666F722074686520536F66744478
:10E7100065766963652E00004368616E67652074E5
:10E7200068652052414D207374617274206C6F6370
:10E730006174696F6E2066726F6D20307825782065
:10E74000746F20307825782E000000004D617869C4
:10E750006D756D2052414D2073697A6520666F7228
:10E76000206170706C69636174696F6E20697320D9
:10E77000307825782E00000073645F626C655F65F9
:10E780006E61626C6528292072657475726E6564AD
:10E790002025732E00000000E31C002030B5144833
:10E7A00091B00078002820D05FF03405ADF84050DB
:10E7B00010A903A861DF30B1052816D011B0BDE85B
:10E7C0003040FBF7CDBA03AC0A49684600F0CAF8FE
:10E7D00007E000BFD0E9002120469047684600F0DE
:10E7E000D8F802980028E1D0F4E711B030BD00005D
:10E7F000E31C0020001E0200F8B5134C2078C0B1C5
:10E800000120A07001F0D4FE112814D0022001F0E4
:10E81000E7FE00258DF800506846FBF73DFB11DF51
:10E82000064625709DF80000FBF75AFB2EB13046D6
:10E83000F8BD0820F8BD0020F8BDA57002F034FB3B
:10E84000032001F0CDFEF6E7E01C00207CB5204C53
:10E85000207808B108207CBD0120A070002001F0C4
:10E86000A7FE112819D0002001F0BAFE1948002691
:10E87000006801908DF800606846FBF70DFB1649B3
:10E8800001A810DF05000AD0002020709DF80000CC
:10E89000FBF726FB2DB128467CBD00207CBD012066
:10E8A000F3E7A67066700721162001F037FE08B165
:10E8B000FBF756FA0721152001F030FE08B1FBF7EF
:10E8C0004FFA02F00DFB012001F08AFEE5E700009F
:10E8D000E01C0020941D0200E59C01000EB50749D4
:10E8E000684600F03FF805E0D0E900108847684628
:10E8F00000F04FF802980028F6D10EBDB01D0200BE
:10E900000148007870470000E01C0020054881782D
:10E9100019B1007818B1FFF76FBF08207047FFF7F3
:10E9200095BF0000E01C00201FB568464BDF30B1EA
:10E93000052814D004B0BDE81040FBF711BA08490F
:10E9400001A800F00FF806E0D0E9002100989047F8
:10E9500001A800F01EF803980028E6D0F4E71FBDD8
:10E960001C1E0200016009684160AFF3008010B511
:10E97000D0E900215368994201D1002104E0D1E996
:10E980000034A34202D01946816010BD08314160B5
:10E99000F0E7816800290BD0026892680A4482601F
:10E9A00041684B689A4203D108314160FFF7DFBFED
:10E9B000704700000C4A10B502F594730EE0991AE6
:10E9C000C91001EBD171491002EBC1010C688442FE
:10E9D00001D90B4602E005D201F108029A42EED3BA
:10E9E000002010BD486810BD301C020000B5FFF7C4
:10E9F000E1FF002800D1014800BD00001C1C0200FE
:10EA00004058002800D00120704708B5002242502D
:10EA10004058009008BD000008480068012110F02F
:10EA2000010F08D14FF0E020E02280F80024C0F868
:10EA30008012C0F8001102480160704700E100E058
:10EA4000180500400649024600200B790BB18520CD
:10EA500070470A6001220A7100224A717047000063
:10EA6000D01B002004490120086004480168C1F35C
:10EA700000410029FAD170470C0000401804004002
:10EA8000002802D00149800108477047391B020065
:10EA90002DE9F0418846054600F09CFF234E0028F2
:10EAA00028461AD0FCF76EFB304490F848008009E5
:10EAB000032802D001280ED007E04FF0A040D0F884
:10EAC0001005E84010F0010F05D003212846BDE8ED
:10EAD000F041FFF773B90221F8E700F087FF002843
:10EAE00022D02846FCF74EFB04464FF4807000EB22
:10EAF00084000F4F81B207EB8400D0F8102542F05C
:10EB00000102C0F810250846FFF788F9B8F1000F98
:10EB10000AD02846FCF736FB56F82000002803D020
:10EB20000120A040C7F80403BDE8F081B021002017
:10EB3000006000402DE9FC41DFF8BC80044608EB92
:10EB40000400002790F930001346C0170E46401C01
:10EB500001D008274CE0B0781946C0F340022046A7
:10EB6000FCF7ECFA0546401C41D0B078410719D4B7
:10EB7000C0070AD04FF0A04000EB8401D1F8000795
:10EB800020F00200C1F8000707E00021737820465A
:10EB900000910A460191FFF7D1F8174920465431F8
:10EBA000FEF7EDFBB078800718D51448317800EBFC
:10EBB0008500D0F81025124B1A40C0F810254FF4EC
:10EBC000F8524FF4403302EA042203EA01410A43B7
:10EBD000D0F810150A43C0F8102509E008EB05002D
:10EBE000327810F8481F41EA8211017000E00427D2
:10EBF0003846BDE8FC810000B021002000600040E4
:10EC0000FFE0FCFF4FF0A041D1F81015C14011F01A
:10EC1000010000D00120704770B5184D95F85800DC
:10EC200008B1082070BD0020411E2A18401CC0B247
:10EC300082F830102028F8D300242046FCF770FA20
:10EC4000641CE4B20C2CF8D300240D49E0206C6560
:10EC500081F8000401264020891FC1F88002C1F814
:10EC600000014FF4BE70FFF7D9F80649F007C1F86C
:10EC7000040385F85860204670BD0000B0210020D4
:10EC800006E000E000600040034890F858000028CB
:10EC900000D0012070470000B02100200121B1EB1D
:10ECA000507F01D10120704700207047002070473D
:10ECB000704700002DE9F0410546164600790F46E1
:10ECC000154A00EBC00102EB810494F8201011B149
:10ECD0000820BDE8F081114951F820102868FFF79D
:10ECE000E5FF08B11120F4E739462846FBF712F991
:10ECF0006660386920601EB1397F2846FDF75CFDEB
:10ED000028680821C0F800150020A061E0610121F9
:10ED1000606184F82010DCE70C2200202C1B02002C
:10ED20002DE9F04704460E460079204900EBC0006B
:10ED300001EB800517463046FFF7B0FF30B12046A3
:10ED400000F036F820B11120BDE8F0871020FBE775
:10ED50006F61AE604FF49076002731462068FFF770
:10ED600054FE4FF4AC7841462068FFF74EFE206811
:10ED7000AA686969C0F84425C0F8481520680121CF
:10ED80008160686878B9B14649462068FFF738FE67
:10ED9000064641462068FFF733FE0643F4D000B133
:10EDA0000F27002068613846CEE700000C220020C3
:10EDB0000079054900EBC00001EB800040690028A4
:10EDC00000D00120704700000C2200202DE9F04700
:10EDD00004460079274900EBC00001EB800720685A
:10EDE0004FF00009C0F80095786880B1206822498A
:10EDF000C0F8081320680121000B40B200F01F0288
:10EE000091404009800000F1E020C0F880112068A6
:10EE1000D0F80C25D0F81485D0F80865D0F8105536
:10EE20004FF0FF31C0F80C15C0F814152068C0F879
:10EE30000815C0F81015501C02D01046FEF7A2FFAE
:10EE4000B8F1FF3F02D04046FEF79CFF681C02D09D
:10EE50002846FEF797FF701C02D03046FEF792FF5F
:10EE60002068FFF725FF87F82090C7F80490BDE8D9
:10EE7000F08700000C2200201003020010B590B1B2
:10EE8000032814D10A480321008801EB004009A19E
:10EE9000FFF7B4F90220FBF7A7FF002807D0BDE871
:10EEA0001040FAF75DBFBDE8104001F0D1BD10BDC4
:10EEB000281D002046617374206164766572746950
:10EEC00073696E672E0000000078002807D104489F
:10EED0003B21008876DF002801D0FAF741BF704758
:10EEE000481B002070B502468888C97B00EB4003B0
:10EEF00002EB4304A41D012901D11188218021883E
:10EF00006288914211D9A5DF012568B111280DD081
:10EF1000FFF76CFD0246064806A1008805EB00409D
:10EF2000BDE87040FFF76EB9657170BD257170BDA9
:10EF3000FC1C002073645F626C655F6761747463BE
:10EF40005F65786368616E67655F6D74755F726534
:10EF5000717565737428292072657475726E6564A5
:10EF60002025732E000000007CB506468D88C888D9
:10EF700005EB450106EB4104A41D172800D217201C
:10EF80002188814200D808466080002020712188B5
:10EF90002846B5DF50B1FFF729FD02460E48012192
:10EFA000008801EB00400DA1FFF72CF960790028E3
:10EFB00010D1F06800280DD01449D1E90201CDE943
:10EFC0000001ADF802506088ADF80400F2686946AF
:10EFD000304690477CBD0000FC1C002073645F62DB
:10EFE0006C655F67617474735F65786368616E6791
:10EFF000655F6D74755F7265706C79282920726524
:10F000007475726E65642025732E0000881A0200E4
:10F0100048B1064A0168914205D140680449401848
:10F0200002D0012800D0032070470000DEC0ADDE12
:10F0300002FEE10E8A7D022A04D90289CB881A4495
:10F04000D21C02814289C988511AC91E4181704768
:10F050002DE9F0410D460221904600F580562980A9
:10F0600000F10804144F1BE031462046FDF71CF95F
:10F0700040B1B8F1000F02D0012288F80020022828
:10F0800016D004E0A0687969884200D978612888A0
:10F0900061880844C01C2880608804EB80040C341C
:10F0A00031462046FDF713F90028DDD1BDE8F08197
:10F0B0004FF480602880F9E7201C002008B500216B
:10F0C000009101460823024A0248FEF73BFD08BDB5
:10F0D000501B0200E81C002008B5002000900448E6
:10F0E0000823044A01680448FEF72CFD08BD00000F
:10F0F000481C0020481B0200E81C00202DE9F05F9E
:10F100000025DFF80891DFF808B12C464FF003081E
:10F11000AA462F46D9F80C0000EB07363046FFF719
:10F1200077FF78B3012847D0032862D100204FF43D
:10F13000806200BF56F82010491C0ED004EB8401F9
:10F140000BEB8102A8F10100566003221FFA80F840
:10F150000BF82120641CA4B24BE0401C9042E9D380
:10F160002C48016879B104EB840102200BF82100DE
:10F170000BEB81014E600881254828304480641CD7
:10F18000A4B205E007E00221066081804FF0010A89
:10F1900045F001052DE004EB840100220BF821204D
:10F1A0000BEB810101F110024E6030460831FFF790
:10F1B0004FFF45F00205CDE7BAF1000F0CD0022059
:10F1C00004EB8401134A0BF821000BEB8101126858
:10F1D0004A60641C0881A4B20E480022011D06602A
:10F1E0003046FFF735FF0B48808802280CD00820F6
:10F1F00005437F1CBFB2032F8CD3B8F1020F00D29E
:10F200000025E8B2BDE8F09F0420F1E7E81C0020EB
:10F2100010240020481C002001494978FBF776BAE9
:10F22000A81B0020002101F013BE30B585B00C46AC
:10F2300005218DF800101546ADF80200FDF7B2F972
:10F24000ADF804006846CDE90245FCF7E5FA05B0E3
:10F2500030BD000070B5054D06460024304655F817
:10F2600024108847641C042CF8D370BDB01A020027
:10F270003EB5104D002400BF05EB041002F064FA07
:10F28000641C022CF8D30124502002210094CDE903
:10F2900001100849084BB039A02201F1A00000F08C
:10F2A000DFFB08B103203EBD0348401E84700020F0
:10F2B0003EBD0000F0200020951B002000F06CB93E
:10F2C00000F06CB970B504460025C168184A28469C
:10F2D00002EB00139B688B4202D102EB001003E0AB
:10F2E000401C0228F4DB00202178082904D00929D9
:10F2F00008D0132914D112E0617A89B980B102F0E3
:10F3000033FA0DE0617A59B950B100218160817BF7
:10F3100041F00201817307490120087003E00125D3
:10F320002046FFF797FF2846BDE8704000F094BFE5
:10F33000F0200020941B002000F0E5B908B51388E8
:10F340009B0000936B4600F05FF908BD002300F0BE
:10F350005BB938B505460024204609E08178284687
:10F3600000F080F810B1052800D003240098401C5C
:10F3700000906946284602F0D3F90028EED134B94E
:10F38000284600F0C4F910B1072802D00324204613
:10F3900038BD0724FBE71346002200F069B90000DE
:10F3A0002DE9F0471F0015460E46814604D0072E72
:10F3B00005D0082E16D102E00E20BDE8F0878DB1F1
:10F3C000022D0FD800F0AEF960B14FF000083146C1
:10F3D000484602F08BF9041E06D0207BA8420DD0CF
:10F3E0000F20EAE70720E8E7FF214FF6FF7002F061
:10F3F0007DF9041E06D0A0F80090A670607BFF285F
:10F4000002D00CE01120D8E72946154800F0FAFA9E
:10F41000014620466173FF2913D04FF00108257380
:10F42000617B0F4800F03CFB02000DD0ABB23146CF
:10F43000384600F007FAB8F1000F0ED0082E05D0BC
:10F440000BE002F081F9DDE70320B6E738886FF0C2
:10F45000050101EB8000796888800020ADE700009D
:10F46000E020002070B5002402F040F905000BD028
:10F47000686820B100F06FF9040000D0032428462A
:10F4800002F072F9204670BD052070BD70B51546BA
:10F490000C46072903D0082C01D0072070BD02F0CC
:10F4A00025F928B105808470BDE8704002F0DCB811
:10F4B000052070BD7CB50D46072903D0082D01D06D
:10F4C00007207CBD002602F011F9040002D060681C
:10F4D00010B11CE005207CBD617B0F4800F0E0FA14
:10F4E00002004FF00000009001908DF8025010D003
:10F4F000237B2946684600F03DF9684602F0A2F8F1
:10F50000211D684600F010F90646092801D0304652
:10F510007CBD03207CBD0000E02000204FF6FF7181
:10F520004180014909680847981A020030B587B040
:10F530001748FCF7FBFA10B1032007B030BDFCF709
:10F5400017FA08B18620F8E700F0CEF90020029003
:10F550004CF2070403900EE0694604A8FCF7B0FAE9
:10F5600000988088A0F5404085B204A8FCF768FAAE
:10F57000284600F075F902AA04A92046FCF787FA8C
:10F580000028E9D00349012008700020D5E70000D9
:10F5900025B80100881B002000F088B900F08CB964
:10F5A00070B586B014460E46054600F03BF940B1F2
:10F5B00005F5404080B20F4A6946FCF768FA40B949
:10F5C00002E0012006B070BD03A96846FCF778FA96
:10F5D00008B10020F6E7A5700398408820800498C1
:10F5E000606003988088A0F5404030806846FCF752
:10F5F00027FAE6E78C1B0020024800214160816069
:10F6000070470000881B0020F0B587B01D461446E7
:10F6100007460E46FF280AD8084600F003F930B125
:10F6200003AA3146384600F0E5F840B902E0072069
:10F6300007B0F0BD01A903A8FCF742FA08B1052004
:10F64000F6E7A67001984088208045B182002868BE
:10F6500090420BD302996068F9F708FF01E0029825
:10F66000606003A8FCF7ECF90020E1E70420DFE785
:10F670007FB586B01E460D460446FF282AD8A878D6
:10F6800000F0D0F830B304F54040ADF80000A878A1
:10F6900003AA00F54040ADF8020068680190288890
:10F6A0000290A978204600F0A5F80528089813D004
:10F6B00010B108A8FCF768FA694603A8FCF724FA19
:10F6C000B0B107281DD0082819D00E2817D0032064
:10F6D0000AB070BD0720FBE728B108AA694603A855
:10F6E000FCF71DFAECE7694603A8FCF714FAE7E714
:10F6F0001EB1314603A8FCF7DAF90020E8E7112033
:10F70000E6E78620E4E74FF6FF7000F0A9B810B5F1
:10F71000FF2801D9072010BD00F0A8F800F02EF84E
:10F72000002010BD00F0F4B870B504460D46807896
:10F7300000F078F858B121882846FCF70DFA002827
:10F7400004D0072805D0092800D0032070BD072069
:10F7500070BD862070BD01B56846FCF715FA00281B
:10F7600000D0032008BD00000149C978FAF7CEBFD8
:10F77000A81B00209BB200F065B8000070B51B4DBF
:10F780008AB00020687000904FF6FF7601903046F6
:10F7900003E0204600F07CF8204600F087F804469D
:10F7A000B0421DD004F5404080B26A4602A9FCF781
:10F7B00076F90A28EDD004F5404080B2FCF798F8BD
:10F7C00008280FD000280BD005461422084905A8A8
:10F7D000F9F74CFEADF8184005A80795FFF79EFE17
:10F7E0000AB070BD01206870FAE70000881B002095
:10F7F0009C1A02007CB5054616460C46084600F0E9
:10F8000011F80020009005F54045019004F54044B2
:10F81000A8B2A1B26B463246FCF732F9002800D0FC
:10F8200005207CBD07280BD0012809D0082807D067
:10F83000052805D0062803D0042801D000207047F1
:10F840000120704710B503EB83034FF6FF7404EA01
:10F8500003138170DB1C99084260018010BD000019
:10F860000149FBF797BC00001021002010B50446A9
:10F87000A0F57F40FF3807D004492046FBF78AFCFB
:10F88000A04201D1012010BD002010BD3021002078
:10F8900010B50446044900F0FBFD03492046BDE8CD
:10F8A0001040203100F0F4BD102100200149FDF787
:10F8B00023BC00003021002070B50A49FDF71CFC74
:10F8C00004464FF6FF7507E000F02CF838B1054903
:10F8D0002046FDF711FC0446AC42F5D170BD204630
:10F8E00070BD00001021002010B508484021F9F734
:10F8F000D6FD4FF480742146044800F0A3F9214658
:10F900000248BDE81040203000F09CB910210020D2
:10F91000FF2803D80146024800F0C3B90020704711
:10F9200010210020FF2803D80146024800F0B9B991
:10F93000002070473021002010B50C46FCF778FB02
:10F94000FF2804D0024900EB400021F8204010BD00
:10F95000401F00201CB500F04FF908B1FAF700FA7B
:10F960000020009001909DF8000020F07E0040F003
:10F970000100303020F080008DF8000007208DF865
:10F98000010010208DF802009DF8030040F00300F4
:10F990008DF803009DF8040040F003008DF804008A
:10F9A000684600F0E3FA08B1FAF7DAF9034800F024
:10F9B000C7FA002801D0FAF7D3F91CBD01FB0100FA
:10F9C0000068012803D0022801D0002070470120E0
:10F9D000704700000449084490F93000082801DB12
:10F9E0000120704700207047B021002004490844DE
:10F9F00090F93000082801D201207047002070479C
:10FA0000B02100202DE9F0410F46060026D03068D5
:10FA100020B3706810B3FF2400251CE029467068ED
:10FA200000F017F948B1FF2C00D12C46281B401CD0
:10FA3000B8420ED12046BDE8F081FF2C06D108E087
:10FA40002146304600F040F8641CE4B2AC42F7D3E3
:10FA5000FF246D1CEDB2B068A842DFD8FF20EAE7B2
:10FA60002DE9F0410400DDE90705069E16D0A9B195
:10FA7000A3B100FB05F7974210D8C21DB6EBD20F19
:10FA80000CD358B155B1E5602160C4E9013081B2B1
:10FA9000184600F0D7F80020BDE8F0810720FBE70A
:10FAA00070B504000D460DD0206858B1606848B1AB
:10FAB000FF2D07D000F0F5F820B1E168206805FBC4
:10FAC000010070BD002070BD70B504000D4611D05E
:10FAD000206800280ED0606800280BD0FF2D09D0C8
:10FAE00000F0DFF8002805D029466068BDE87040C6
:10FAF00000F0E3B870BD002901D000F0CDBF704721
:10FB0000F8B5044600781E4D03260E281DD2DFE806
:10FB100000F0071C0F1C1D1C24351C331C352E3512
:10FB2000288818A106EB0040BDE8F840FEF766BB48
:10FB30006088FAF7D7FD0246207A0090288863880B
:10FB400006EB00401AA1FEF76CFBF8BD0020009008
:10FB500060886946FFF7CFFFF8BDFBF7EBFE08288A
:10FB6000FAD00028F8D0BDE8F840FAF7F9B8BDE8B7
:10FB7000F8400020FAF712B82069F2E7A068F0E731
:10FB8000281D0020436F6E6E656374656420746F7A
:10FB900020612070726576696F75736C7920626F71
:10FBA0006E646564206465766963652E00000000FC
:10FBB000436F6E6E656374696F6E207365637572F3
:10FBC00065643A20726F6C653A2025642C20636F5F
:10FBD0006E6E5F68616E646C653A20307825782CB3
:10FBE0002070726F6365647572653A2025642E001B
:10FBF000FBF7EEBDFBF7ECBD10B5FFF797FC88B93E
:10FC0000FFF736FB70B900F049FF58B901F064F80E
:10FC100040B9FCF7A9F928B9FCF78EFA10B9FCF73E
:10FC200031FC08B1032010BD05484FF6FF718180FB
:10FC300000218160417001210170002010BD000091
:10FC4000981B0020002803D0C91DC908F9F727BC5C
:10FC50007047002809D001F0070301229A40D2B270
:10FC600000EBD1001146FCF7E1BF70472DE9F041F0
:10FC70000D46060013D0002401270EE004F0070013
:10FC800007FA00F0C1B206EBD400FCF7CFFF10B1C9
:10FC90002046BDE8F081641CA4B2AC42EED32846F5
:10FCA000F7E740B100EBD10001F007020078012135
:10FCB0009140084000D001207047F8B50400C1F31E
:10FCC000C70501F007014FF0010000FA01F0C6B2CC
:10FCD0000FD0605D30420CD000208DF800006846E7
:10FCE000FAF7DAF8605DB04360559DF80000FAF766
:10FCF000F7F8F8BD2DE9F041044686B00127808869
:10FD0000FCF78EFB6080207800263F4D082808D045
:10FD1000092820D04FF6FF780A2829D00B2853D184
:10FD200058E0607A10B1012809D04DE0A86830B1E0
:10FD3000E168814203D1AE60A088A88016E06878AF
:10FD4000E8B3A088A98888423ED1207A06283BD112
:10FD500000F066FA38E0607A88BBA86878B3E1689A
:10FD6000814231D1AE60E868401EE860E6602BE079
:10FD7000A878E8B14046FFF7A3FA4146404517D1BD
:10FD80000846FFF79BFA404512D1AE701421684631
:10FD9000F9F785FB0C208DF80000ADF80480ADF874
:10FDA000028000272046FBF713FD6846FBF710FD95
:10FDB000687838B1A088A988884203D100E003E0C0
:10FDC00000F02EFA002F1CD006B02046BDE8F0410E
:10FDD000FBF7FEBCA8780028F6D0AE701421684668
:10FDE000F9F75DFB0D208DF80000ADF80480ADF84B
:10FDF0000280A06802902046FBF7EAFC6846FBF709
:10FE0000E7FC06B0BDE8F081981B002003490978A3
:10FE100009B1FCF7B3BB082070470000981B002015
:10FE20002DE9FF4F2A4883B09946007892468B46C9
:10FE3000B8B14FF6FF763046FFF742FA8046002011
:10FE40000090244801AA062100680190CDF808D04E
:10FE50004046FFF773FA00256C1E3746072804D08A
:10FE600017E0082007B0BDE8F08F0520FAE7002072
:10FE70000090A84201D305464746A04201D204465D
:10FE800046464046FFF71CFA804601AA0621FFF7C6
:10FE900055FAD8B10528EAD0A8F57F41FF3901D03D
:10FEA0000320DFE70399002001B10F80BBF1000FB1
:10FEB00001D0CBF80050BAF1000F01D0AAF80060D1
:10FEC000B9F1000FCED0C9F80040CBE70098D0E7D9
:10FED000981B0020C01A020070B5184E86B030780A
:10FEE000D0B10120B0704FF6FF742046FFF7E8F95B
:10FEF0000546A0421DD10020B07014216846F9F7D4
:10FF0000CEFA0C208DF80000ADF80440ADF80240A8
:10FF10006846FBF75DFC0EE0082006B070BD00BF30
:10FF2000FFF774FF08B10320F7E72846FFF7C8F989
:10FF30000546A542F4D10020EFE70000981B002001
:10FF4000084A117821B1D178032903D304207047DE
:10FF500008207047044B43F82100491CD170002051
:10FF600070470000981B00205021002003490978A9
:10FF700009B100F0E5BD082070470000981B002083
:10FF8000002801D0FBF724BC7047000010B50C46D8
:10FF9000017A052908D0407A38B1084808A10268DA
:10FFA0002046FDF759FB00E01AB106A12046FDF7F7
:10FFB00053FB2046BDE81040FDF75BBBBC1C002096
:10FFC000257300000D0A000038B5C3880D460446AD
:10FFD00033B114A0009015A216A12846FDF73CFBF2
:10FFE000217A05291CD0607A48B1A088FDF7D0FF9E
:10FFF000164951F8202016A12846FDF72DFBA088B0
:020000040002F8
:100000000021FEF7A3F903461049207A143951F86C
:10001000202001B02846BDE830400EA1FDF71CBBF2
:1000200038BD00001B5B306D000000001B5B313BE6
:1000300033316D0025734C6F67732064726F70707D
:100040006564202825642925730D0A00BC1C002046
:10005000257300003C25733E2025733A20000000E4
:100060000146054810B50068FDF779F804461C21E3
:10007000F9F715FA204610BD401B02000146024860
:100080000068FDF78DB80000401B020003480249DC
:100090000068FDF76FB80000681C0020C81B020054
:1000A000F0B5254D254E85B004460027686828B96F
:1000B000214930680831FDF768F86860014600782A
:1000C000072817D2DFE800F0160408080E0E120009
:1000D0002046FCF7AFFA02E0204601F0CFFB040017
:1000E00028D008E02046FBF7D5F9F8E72046FBF7D3
:1000F000E5FDF4E70F2414216846F9F7D0F9A4F5DB
:10010000E8501D3800D10024019469466868FBF767
:10011000A3FA6846FBF7DAFA07496F600024083152
:100120003068FDF727F8044801210C30FDF7C7F8C7
:100130000028BBD105B0F0BD201C0020401B0200F0
:100140002DE9F041234C0025234E207A012730B9B8
:100150002248311D0068FDF718F8306038B10220E0
:1001600020723168087928B101281ED116E0656037
:10017000BDE8F081D1E90503C01A4FF480529042E6
:1001800000D31046B7EB900F01D2820800E00122A5
:100190000869C9681844194429DF03E0D1E903015B
:1001A000084428DF58B1112812D003213068FBF72A
:1001B0009DFA25726560BDE8F041FFF767BF207CBE
:1001C0000028D5D1BDE8F04100210220FDF768BC30
:1001D0002772CDE7D4240020641C0020C81B020035
:1001E00010B501210448FDF750F8002803D1BDE8FF
:1001F0001040FFF755BF10BD2C1C002010B5074C58
:10020000201DFDF733F8002806D1607C002803D1BB
:10021000BDE81040FFF794BF10BD0000D4240020BB
:10022000084910B500231A46A1F10800FFF7F8FDB0
:1002300030B1052804D0002002490C39487010BDA7
:100240000120F9E7A41B002010B510461A46F9F763
:100250000DF9002010BD00002DE9F0471B4F82462C
:100260000026387886B0002821D00024DFF860808E
:10027000A14600BF08EB0415A87B810702D410EA51
:100280000A0F1BD00126284601F0EEF9B0B14FF657
:10029000FF71ADF802102988ADF80410862809D046
:1002A00007218DF8001002906846FEF7D3FF06B0D4
:1002B000BDE8F08706208DF80000F5E7641C022CED
:1002C000D8D3002EF3D187F80090F0E7941B0020DC
:1002D000F02000202DE9F04707461E481C46154631
:1002E00000780E4670B185B17CB1DFF86C804FF0BC
:1002F0000009A08802282BD200EB800118F8210009
:1003000010BB19E00220BDE8F0870520FBE720685C
:100310001FB181883A8891420ED11EB1018832887E
:10032000914209D180682860206868600A482830B6
:10033000008928810020E6E7A088214600F05EF8C9
:100340000028E4D1C4F80090A088401CA080D0E729
:100350000A20D8E7401C002010240020F8B50546EC
:100360004068244F0C46002648B32349CA6882429D
:1003700025D80969814222D3FCF7B8FAF8B1288957
:10038000398988421BD1D5E900018A68904216D18B
:100390000020A7F1280200BF00EB800302EB8303DB
:1003A0005B688B4205D203F580538B4201D92080D4
:1003B00011E0401C80B20228EED30020F8BD268058
:1003C00000960AE0009829688068884205D1009864
:1003D0006860388928810120F8BD2088694600F0CE
:1003E0000DF80028EED12088401C80B22080022821
:1003F000E6D3E2E738240020E81C002070B50E4662
:1004000000EB8001134800EB81004468306804F57C
:10041000805518B1418800EB810411E0083410E0E8
:1004200029462046FBF740FF20B1012805D00228CD
:1004300007D10DE00120346070BD608804EB8004BA
:100440000C3429462046FBF742FF0028E8D170BD56
:10045000002070BD1024002038B50C46002100910A
:1004600001460423074A0848FDF76CFB08B10E203B
:1004700038BD064A04EB840102EB810101200874B7
:10048000002038BD441B0200E81C0020102400207E
:100490000A46FF2803D801461046FFF70EBC7047F6
:1004A0000846704770B5012670044FF0E021002522
:1004B000C1F88001084C4010C4F84803C4F8080390
:1004C00066602F20FEF7DCFAA660044C2F20A560A2
:1004D000FEF7D6FAA57070BD00100140F81B002091
:1004E0001FB501238DF800308DF808100192D0E976
:1004F0000012684690471FBD10B504460648417972
:100500002046FAF703F9002804D12046BDE8104040
:1005100000F014BA10BD0000701B002070B50D462D
:100520000446F9F7DDFA70B12846F9F7EBFA68B13D
:100530006807000E002C0CDA04F00F0101F1E02135
:1005400081F8140D09E042F2010070BD42F2020090
:1005500070BD04F1E02484F80004002070BD0000A8
:1005600038B50021012548B101280CD0032809D154
:10057000FEF752FABDE83840FDF736B84FF0E020FC
:10058000C0F8805138BD8DF800106846F9F784FC3A
:10059000064C207808B9FDF70BF8E068401CE060D5
:1005A000A5709DF80000F9F79BFC38BD9C21002048
:1005B0003EB5044609496846FEF7D4F908E000BF95
:1005C000D0E900212046904730B16846FEF7E1F9B6
:1005D00002980028F4D13EBD11203EBD981D0200B6
:1005E0003EB5044608496846FEF7BCF907E000BF7F
:1005F000D0E90021204690476846FEF7CAF90298E4
:100600000028F5D13EBD0000A41D02002DE9FC41EB
:1006100004460C3000278046FBF7D4FF4FF6FF75E9
:100620000646A842208803D1FBF7BCFF064602E03D
:100630003146FBF7A1FF20880022012100F0C6F817
:10064000AE4212D06A4607213046FEF77FFE60B9FF
:10065000019D95F844003435C00705D1414605F1A8
:100660001200FBF774FF00B12F46002320881A46C2
:10067000394686DF05000BD0002320881A46314614
:1006800000F088F82088294600F002F9BDE8FC81D6
:10069000002FFBD1002320881A46314600F07AF85B
:1006A0002088002241F20601FAF7AAFFEEE70000D7
:1006B0002DE9FC411D46089C16460F46804644B174
:1006C0006B46012207213846FEF76AFE112801D049
:1006D00010B10320BDE8FC8150210198F8F7DFFE3E
:1006E000019806700198E560343020600198183058
:1006F00020610198401C60610748E0610199404613
:100700001131FBF711FE0028E3D107213846FEF72F
:10071000D1FE0528DDD0DDE75C210020002835D0A2
:100720000278910701D411062FD4C2F302110429D3
:100730002BD8930703D5032901D1110625D543787A
:1007400081788B4221D8072B1FD310291DD8C1785F
:100750004B071AD40079430717D40B0715D40307A6
:1007600013D4D2074FEAC17201D042B10FE062B98F
:1007700089070AD4C10708D1800706D407E0890792
:1007800005D4C10703D1800701D4002070470120A0
:100790007047000070B50C4605466AB1002B12D0B8
:1007A00009480122C1782846F9F7C8FF21462846A2
:1007B000BDE87040FBF7E0BE002B04D0BDE8704000
:1007C0000846FBF7DBBE70BDA81B0020F0B5174D37
:1007D00014460F460A4685B006462978F9F7AEFF5B
:1007E000002F1FD00CB1012200E0002269783046B2
:1007F000F9F7A4FF012C17D00022A9783046F9F7A9
:100800009DFF0022E9783046F9F798FF1422084945
:100810006846F8F72BFEADF802608DF80840684690
:10082000FAF7ECFF05B0F0BD0122E6E7A81B0020B7
:10083000D41A020010B586B0044614216846F8F7B1
:100840002EFE04208DF80000ADF802406846FAF74D
:10085000D5FF06B010BD000002498969002900D00B
:1008600008477047AC1E002030B585B00C460546E1
:10087000142206496846F8F7F9FDADF802506846BB
:100880000294FAF797FF05B030BD0000181A020075
:1008900030B585B00C460546142206496846F8F77F
:1008A000E5FDADF8025068460294FAF7A7FF05B0DF
:1008B00030BD0000E81A020010B5094C0020D2B289
:1008C000207004F10800FEF72BFA08B1F9F748FA96
:1008D0006078002802D021780029FAD010BD0000ED
:1008E000741C00200348002201490079F9F7E4BE96
:1008F000F9040200701B00207CB50E490E4C00224A
:10090000D1E90001CDE900016946A088FEF743FD69
:100910004FF6FF7507E00846FEF7D2FCA0800022E4
:100920006946FEF738FDA188A94201D01128F2D10D
:100930007CBD00006C1A02007C1B002070B586B0E4
:10094000064601250024FBF793FC112812D005DC94
:10095000F0B1062828D0082808D125E0A0F540519C
:10096000023907D0A1F54071FF3924D00146304645
:10097000FFF77AFF2A46124D30462979F9F7DEFE55
:10098000697906B022463046BDE87040F9F7D6BE18
:1009900014220C496846F8F769FDADF8026001249D
:1009A0006846FAF707FFE5E700253046FBF7FAFD52
:1009B000FBF7B4FBDEE73046FCF7FCF8DAE70000B3
:1009C000701B0020401A02002DE9F0410746806AA2
:1009D00014468846C8B3002531E000BFB96A05EB6C
:1009E000450001EB8006B088801CFE2802D90C204F
:1009F000BDE8F0812288401C08F8020020881622F9
:100A0000401C80B2208008F800202088401C80B262
:100A1000208000EB0801308800F07CFC218808442D
:100A200080B22080B28842B1B16871B14044F8F719
:100A30001DFD2088B188084420806D1CEDB297F818
:100A40002C00A842CAD80020D2E7FFE70720CFE752
:100A500010B50020FAF7C8F908B1F9F781F9FAF7EB
:100A60001DF908B1F9F77CF933DF002803D0BDE8A0
:100A70001040F9F775B910BD10B500F0ABF8054896
:100A8000002203494078BDE81040F9F715BE000088
:100A900091CA0100B01B002000F016B910B5114832
:100AA000FBF7A9F80F48401CFBF7A5F80D48801C80
:100AB000FBF7A1F80B48C01CFBF79DF80948001D87
:100AC000FBF799F80748401DFBF795F80548401ECD
:100AD0008179182903D00121C171002010BD0320A4
:100AE00010BD0000B11B002010B50078114C0A2881
:100AF00013D004DC082810D009281AD10DE00B28E7
:100B00000BD0132815D100220B49A079F9F7D4FD99
:100B100000220A49A078F9F7CFFD00220649607942
:100B2000F9F7CAFD6078BDE8104000220349F9F7E3
:100B3000C3BD10BDB01B002025F2010091CA010009
:100B400070B50B4C05004FF001060CD0FFF7E6FD29
:100B500058B1286820612879207504F11000A06040
:100B60002670002070BD0020F9E7072070BD00004E
:100B7000B01B002010B504460078052802D01228CA
:100B800021D105E06088A168BDE8104000F060B99F
:100B90000F480021806880B10D48237A103000781A
:100BA00000F0010203B101239A4206D3627AC0F336
:100BB000400002B10122904200D20121608801234D
:100BC0000022FBF7C3FE2046BDE81040FAF724BE22
:100BD000B01B002030B50446008885B014284FD0E3
:100BE0000ADC11282CD0132828D134F8040FF9F787
:100BF00079FD01282FD038E0192847D01A281DD1B7
:100C0000A088FEF709FB002818D1A088F9F744FD59
:100C10000028A0884BD02A4900220978F9F78EFDD8
:100C200002208DF80000A088ADF8020000208DF8A9
:100C300008008DF809006846FAF7E0FD05B030BD00
:100C4000207A3D2804D04FF48851A088002224E067
:100C500041F23D01F9E72079C00701D0012200E00F
:100C6000022220880121FFF7B1FD34F8045B142231
:100C700014496846F8F7FAFBADF802500294DAE737
:100C800005B0201DBDE83040FFF7C0BC217A201D13
:100C900041B14279008802F0030205B0BDE830405E
:100CA000FBF7B0BE05B0BDE83040F9F779B905B043
:100CB0000122BDE8304041F20601FAF7A1BC000074
:100CC000A81B0020101B02000A7802490979F9F7D5
:100CD00035BD0000A81B002010B51448FAF782FFAC
:100CE0001248401CFAF77EFF1048801CFAF77AFF82
:100CF0000E48C01CFAF776FF0C48001DFAF772FF89
:100D00000A48017818290FD0417818290CD0817829
:100D1000182909D0C178182906D00179182903D0DB
:100D200001214171002010BD032010BDA81B00202F
:100D300070B50C460546F9F7D5FC012802D043F200
:100D4000020070BD21004FF00000FAD028467EDF7F
:100D500070BD00002DE9F74F8AB0924688460A9888
:100D6000F9F7C0FC06464FF6FF7900244D462746AA
:100D70000A98FEF7F9FC8346202101A8F8F78FFBBB
:100D8000012E01D0DEB105E02F48002201790A983A
:100D9000F9F7D4FCB8F1000F16D098F80000C0079E
:100DA00014D00A98FBF7FEFB0546484516D1FEF71E
:100DB000C3FA054648450ED04FF0010B0CE043F254
:100DC00002000DB0BDE8F08F852721E01F48CDF867
:100DD00010A008901CE003246CB121E0012E0AD180
:100DE0000A98F8F72BFF30B90A98FFF723FD0A9805
:100DF000F8F724FF50B101A8009053463246294627
:100E00000A98FFF755FC040002D009E0852712E09C
:100E1000012E10D001AB002239460A987FDF04462C
:100E200054EA07000DD000225B4629460A98FFF7D6
:100E3000B1FC2046C5E701AB424639460A987FDF40
:100E4000EDE70122F0E70000A81B00205C21002054
:100E50003EB505460C466846FCF744F96A4621460D
:100E60002846FEF7E2F909480099C2682846FFF7CC
:100E700071FF0446014601222846FAF7D9FE2146B1
:100E80002846009AFAF75CFC3EBD0000B01B00202B
:100E9000002805D10349012048700020FAF796B9CF
:100EA000704700009C21002010B51620F8F718FEAE
:100EB00048B10A4882684FF4800152B1016821F4B8
:100EC0008001016010BDBDE8104042F20100F8F75A
:100ED00047BF4FF0E020C0F8801110BD5C23002018
:100EE00010B51620F8F7FCFD80B10F4890F800040B
:100EF0004009F8F707FE60B10C4882684FF48001A2
:100F00006AB1016841F48001016010BD42F2010044
:100F100001E042F20200BDE81040F8F721BF4FF0B7
:100F2000E020C0F8001110BD16E000E05C230020B6
:100F30002DE9F84F204D92468946064698460122F3
:100F400069461846AF68FAF785F858B3009800214B
:100F50000446801C09E000BF00EA07035AF821207C
:100F600005EB8303401C491CDA604145F4D34FEA8A
:100F7000164AFAF71BFB4AEA0041601C384005EBB1
:100F800080003C4005EB8402C160D06866F3C50078
:100F900068F3891069F39F2020F00300401C20F0C3
:100FA0000400D06095F8200402E000BFFDF716F8B9
:100FB0000028FBD1BDE8F88FF42500202DE9F84F7B
:100FC0001D4C00256846D4E901A6FAF7F9FA002776
:100FD00038B30023009A61681CE0D1F800C00846CD
:100FE000944503D9ACEB02020A6015E0A2EB0C02B7
:100FF00063440760D0F80CC0C1698146BCF1000FA2
:1010000008D006EB030828F07F48C0E9018CC9F836
:101010001C5005460029E0D128466160FBF74EFDD3
:1010200003E02846FBF74AFD10B15046FAF7F0F806
:10103000E770BDE8F88F0000F81B00200D4B10B5DD
:10104000596831B102680C68A24204D8A21A0A6039
:10105000C161586010BD0B4603E00B46C969121B05
:1010600021B10C689442F8D3A41A0C600260C161EB
:10107000D86110BDF81B00202DE9F041144E7768AF
:101080003D462C4603E0844204D02546E469002C0A
:10109000F9D11BE0D4B1A5420BD1F869706040B919
:1010A0000C49012088600021B160F0702F20FDF70D
:1010B000E7FC2168E069E86110B102681144016051
:1010C0007068874202D00120BDE8F0810020FBE774
:1010D000F81B0020001001407CB5064600240D4698
:1010E0008DF800406846F8F7D7FE01A800F0E4F953
:1010F00070B10570094946609DF8040048709DF87C
:101100000000F8F7EDFE1420F8F7FEFA20467CBD4B
:1011100004249DF80000F8F7E3FEF7E750220020D2
:101120002DE9F041194D6C68002C2CD0184800278F
:101130000068A968B846401A20F07F462068B0428F
:101140000CD82146361A0744E469087C20B181F89E
:101150001080886949698847002CEFD12978687820
:10116000814206D1401CC0B26870022801D185F8C6
:101170000180064869780C3040F82170BDE8F041E4
:101180001420F8F7C1BABDE8F0810000F81B002078
:10119000041501400149012008707047741C0020AB
:1011A00010B588B0044620220E496846F8F75EF96B
:1011B00006200090C01F0190029003904FF0EB704A
:1011C00006900CB1084A00E0002269460748FCF787
:1011D00023FA08B1F8F7C4FD0448001F447008B0B2
:1011E00010BD0000641D020095110200781C002053
:1011F0001FB50A4601788DF8001041680191017A07
:101200008DF80810C0680390044850F82210001FA1
:1012100050F82220684690471FBD0000CC1B0020DC
:101220002DE9FF410C464FF4927705463946FDF70C
:10123000E7FB0026C0B139462846FDF7E6FB022051
:101240008DF80000D5F88004C5F880040390D5F827
:101250003C058DF80800E0680190A661E661D4E9DC
:1012600000126846904723E04FF4887739462846B5
:10127000FDF7C6FBE0B139462846FDF7C6FBD5F8B9
:101280003C15A069884213D1E06960B1E268D5F8E5
:10129000000220F02000C5F80002E069A06120698A
:1012A000E661E06001E0A661E2682046FFF718F918
:1012B0004FF4A27739462846FDF7A2FB60B13946C4
:1012C0002846FDF7A2FBA06930B1A661D5F83C1510
:1012D0002046E268FFF704F94FF490773946284634
:1012E000FDF78EFB002813D039462846FDF78DFB0D
:1012F000606900280CD0D5F84C058DF800608DF899
:101300000800A06801906661D4E900126846904721
:10131000BDE8FF810870000A487002207047000095
:1013200010B514210448F8F7BAF804480068FBF730
:10133000FBFE002010BD0000D4240020C81B0200CA
:101340002DE9F05F8346DDE90A4A994690460D464D
:101350000846012703E000BFB0FBF8F07F1C4045C2
:10136000FAD2B94500D94F465FEACA7012D18CB1A2
:101370005FEA8A7002D5B9F1000F01D0202607E09C
:10138000302605E031465846641EF9F7ABFE0CB135
:10139000A742F7D35FF00106B9F1010F02D9A9F115
:1013A000010903E0B5FBF6F0404502D306FB08F661
:1013B000F2E7DFF83C9000BFB5FBF6F000FB1655F6
:1013C00019F800105846F9F78DFEB6FBF8F6002E16
:1013D000F2D15FEACA7009D0002C07D0A74205D22B
:1013E00020215846641EF9F77DFEF5E7BDE8F09F21
:1013F000581B02000348002201498078F9F75CB9C4
:1014000015B40100701B0020F8B5054680B2FBF74B
:1014100075F9040013D0154E207A0027317B8842DD
:101420000ED2A8B204F10A0175DF28B1112806D046
:10143000BDE8F840FFF710BA207A401C2072F8BDD2
:101440002772307C38B1A8B23B2176DF18B108286A
:1014500001D0FFF701FA71690029F0D08DF8007012
:10146000ADF8025068468847F8BD0000AC1E002069
:10147000417939B190F8B21021B990F8B40008B1AF
:10148000012070470020704701460148FBF7D3BE9A
:10149000C81E002030B40446007A00280AD06088B4
:1014A000002166DF28B1112802D0616830BC0847EE
:1014B0000120207230BC70470A494A788B78521C50
:1014C000D2B2934200D100220B78934201D1002086
:1014D00070470270487800EB400001EBC000001D2F
:1014E00070470000502200202DE9FC411646DDE93E
:1014F0000854CDE900541F468046022200F00CF843
:10150000002807D1CDE900543B4610223146404621
:1015100000F002F8BDE8FC812DE9FC5F0026DDE962
:101520000C4B994692468E4680462788354630E0D9
:10153000D8F80400002200EB85006946006801909D
:1015400001A864DF002830D19DF8000050451FD16C
:101550000EB1002100E002212288084411185945EB
:1015600022D846B9521C90B2208009F800E02088A9
:10157000401C20800126218801A801EB0902694650
:1015800064DF002811D120889DF8001008442080D5
:101590006D1CB8F80000A842CADC56B12088C01BF8
:1015A000401E80B2FF2802D90C20BDE8FC9F09F83C
:1015B00007000020F9E710B5042817D209B1032469
:1015C00000E00024F9F7B8FA4FF0A04101EB8000E9
:1015D000D0F8001721F44031C0F80017D0F80017F8
:1015E00041EA0441C0F80017002010BD062010BDDC
:1015F000002070472DE9F84F114D884681461E4660
:1016000017466946DDF828A02868FBF7A8FD040006
:1016100013D01C21F7F743FF00202071C4F800907D
:10162000C4E90486C4E902A769462868FBF7B8FD47
:10163000FEF7E4FD0020BDE8F88F0420FBE7000082
:10164000C81B020082780121012A0BD0062A09D08A
:10165000072A06D0082A06D14168898809318908F5
:1016600000E01421018070471CB504460020009062
:101670000190A0788DF80200617B1A48FEF710FAFD
:10168000020017D0237BA1786846FEF773F86846FE
:10169000FFF7D8FF208804F1080369466268FDF768
:1016A000E7FF48B1072806D001210F4A112808D0CA
:1016B00086280FD003201CBDA17B21F00301A1735C
:1016C0001CBDA07B20F0010040F00200A07311704F
:1016D00000201CBDA37B23F0020343F00103A3738E
:1016E00011701CBDE0200020941B002038B5054679
:1016F0000C46002001E00098401C009069462846F6
:1017000000F00EF800280AD08178A142F3D1817B45
:101710008A07F0D4C907EED181680029EBD138BD22
:1017200010B5084B0A6809E003EB021424888442D0
:1017300003D103EB02100A6010BD521C022AF3D33E
:10174000002010BDF02000204FF6FF710180FF2126
:1017500081704173817B21F003018173002101734A
:10176000416081607047000070B50546002406E0C6
:10177000687B2044C1B20648FEF7A6F9641C287BAA
:10178000A042F5D82846BDE87040FFF7DDBF000055
:10179000E02000202DE9FC470646364898461446CE
:1017A00000780D464FF0000978B37DB32888A0F586
:1017B0007F41FF3931D0688848B36868FBF796F8F5
:1017C00068B374B32088ADF80000678801A8FEF7FD
:1017D00047FC04002FD084F800804FF0000A84F802
:1017E00016A0BDF80000A082686820612148012190
:1017F0000C38FBF73EFDE060288820816888A080D7
:10180000E780B8F1030F1DD020E001E003E004E021
:101810000220BDE8FC870520FBE70420F9E7032050
:10182000F7E7FFE72889694687B2384600F0ACF849
:101830000028EED1CAE7BDF80010384600F098F84D
:101840000820E6E70420A0753068A061A4F80A909B
:1018500001A8FEF713FC46B1C6F804A0E1680648EB
:10186000316086F80AA000893081FEF7B9FC0020BB
:10187000CFE70000401C0020382400202DE9F84369
:101880000D46898A374A01EB810102EB810630B1AE
:1018900029463046FDF7CEFB0120BDE8F8833189AB
:1018A0007068002400EB81072E48A97DA8384FF00E
:1018B0000E0807294ED2DFE801F00D2D1624044052
:1018C0004A004460A969016026482749A838FEF704
:1018D00045FD30B10220A875042339462A1D009425
:1018E00023E00A20D9E728692A4608B1032000E04E
:1018F00001209075042305F10C0207F10801009402
:1019000013E00120A8750094E88807F10C0183001A
:101910002A690AE028782A4603280CD00620907508
:10192000042305F10802391D00941048FCF70AF958
:10193000A8B144460FE00520F1E70621A9750A4940
:1019400040680988FEF788FD040004D107E041F6ED
:101950001D5400E00F2429463046FDF76BFB20465E
:101960009BE7000010240020201C0020E81C002021
:1019700001EB8102034901EB82014A89101AC01E62
:10198000488170471024002070B5C01C82B240F21C
:10199000FE30824201D3092070BD114B00204FF46C
:1019A000806500BF00EB800413F8246096B903EB58
:1019B00084063489768914443444A4B2AC4209D2F2
:1019C000088000EB800003EB8000418911444181D5
:1019D000002070BD401C80B20228E3D3072070BDF8
:1019E00010240020111213140D0E0F100C1E0020D5
:1019F0002C1E0020581E00200D000300BDAC01006D
:101A00000E000300BDAC01000F000300BDAC0100DF
:101A100010000300BDAC0100070000000000000042
:101A200000000000000000000000000006000000B0
:101A300000000000000000000000000000000000A6
:101A40001000000000000000000000000000000086
:101A50000000000011000000000000000000000075
:101A60000000000000000000010000000100010073
:101A7000681A0200010001007C1A02000000000048
:101A8000F5FB010039BF0100770A000000000000EB
:101A9000770A000000000000C5F201000700000006
:101AA0000000000000000000000000000000000036
:101AB000F5FC0100E90A020039C20100B9BF0100CA
:101AC000010000000000000001000600A41B00202F
:101AD000750B020001000000000000000000000083
:101AE00000000000000000000700000000000000EF
:101AF00000000000000000000000000003000000E3
:101B000000000000000000000000000000000000D5
:101B100005000000000000000000000000000000C0
:101B20000000000081FF010000000050B19A010098
:101B300003000000302200200738FDD87047000065
:101B40000C1C00200000FFFFDEC0ADDEFF011EF117
:101B5000DEC0ADDEFE011EF13031323334353637B2
:101B600038394142434445466E72665F6673746F0E
:101B7000726167655F696E6974006E72665F667335
:101B8000746F726167655F756E696E6974006E72FD
:101B9000665F6673746F726167655F72656164002A
:101BA0006E72665F6673746F726167655F77726984
:101BB0007465006E72665F6673746F726167655FED
:101BC0006572617365000000501C00200010000069
:101BD000040000000100000001C601002113020002
:101BE00049020200F51502000DB60100A104020031
:101BF000F115020085C8010000000000000000008F
:101C000000000000000000000000000000000000D4
:101C1000F81B0200101C020004000000556E6B6EE1
:101C20006F776E206572726F7220636F646500005B
:101C300000000000782202000100000024210200C0
:101C400002000000181F020003000000982102009B
:101C500004000000EC21020005000000CC2002007E
:101C6000060000006820020007000000D4210200E6
:101C700008000000E02002000900000044210200EA
:101C80000A000000602202000B000000001F02009A
:101C90000C000000F82002000D000000C822020025
:101CA0000E000000C42102000F000000002202000C
:101CB000100000003422020011000000DC220200AB
:101CC00012000000B0220200130000004C220200AB
:101CD000800000008020020081000000BC1F020084
:101CE000820000007C1F0200830000005C1F0200D5
:101CF00084000000981F020085000000A42002005C
:101D000086000000AC210200900000004820020084
:101D1000910000003C1F0200920000000C21020014
:101D200000820000142202000182000060210200F3
:101D3000028200007C21020000840000D81F020003
:101D4000018400008422020002840000202002009E
:101D500003840000FC1F020079DF010061DF010045
:101D600059DF0100FFFFFFFFFFFFFFFFFFFFFFFF46
:101D7000FFFFFFFF00000000000000000000D60190
:101D800007000000742602007C260200000000000C
:101D90000000000001000007841D0200941D0200E5
:101DA00008000000BC1D0200CC1D0200080000005D
:101DB000CC1D0200DC1D020008000000A426020069
:101DC000B42602000000000000000000942602007B
:101DD000A4260200000000000000000034260200DB
:101DE0003C2602003C260200642602006426020013
:101DF0006C2602006C26020074260200481B00209C
:101E0000DC1D0200FC1D0200080000007C26020010
:101E10008C2602008C260200942602000C1E020072
:101E20001C1E0200080000000040404040404040AE
:101E3000404041414141414040404040404040409D
:101E40004040404040404040400502020202020241
:101E50000202020202020202022020202020202090
:101E600020202002020202020202909090909090A4
:101E70001010101010101010101010101010101062
:101E800010101010020202020202888888888888D6
:101E900008080808080808080808080808080808C2
:101EA000080808080202020240000000291E020081
:101EB000616464725F69735F77697468696E5F6299
:101EC0006F756E647328705F66732C207061676530
:101ED0005F616464722C20286C656E202A20705F1C
:101EE00066732D3E705F666C6173685F696E666FC6
:101EF0002D3E65726173655F756E697429290000F6
:101F00004E52465F4552524F525F494E56414C49E0
:101F1000445F4441544100004E52465F4552524F87
:101F2000525F534F46544445564943455F4E4F54C4
:101F30005F454E41424C4544000000004E52465F12
:101F40004552524F525F464541545552455F4E4FA0
:101F5000545F454E41424C45440000004E52465F9E
:101F60004552524F525F4D555445585F554E4C4F58
:101F7000434B5F4641494C45440000004E52465F8A
:101F80004552524F525F4D555445585F4C4F434B4D
:101F90005F4641494C4544004E52465F4552524FC0
:101FA000525F4D555445585F434F4E445F494E492B
:101FB000545F4641494C4544000000004E52465F84
:101FC0004552524F525F4D555445585F494E495402
:101FD0005F4641494C4544004E52465F4552524F80
:101FE000525F424C455F495053505F52585F504BCF
:101FF000545F5452554E4341544544004E52465F3F
:102000004552524F525F424C455F495053505F50CA
:102010004545525F52454A4543544544000000003F
:102020004E52465F4552524F525F424C455F4950B7
:1020300053505F4C494E4B5F444953434F4E4E45BE
:1020400043544544000000004E52465F4552524FF3
:10205000525F4150495F4E4F545F494D504C454D82
:10206000454E5445440000004E52465F4552524F83
:10207000525F4E4F545F535550504F525445440099
:102080004E52465F4552524F525F4D4F44554C455C
:102090005F4E4F545F494E495449414C495A45445B
:1020A000000000004E52465F4552524F525F4D4F66
:1020B00044554C455F414C52454144595F494E4956
:1020C0005449414C495A4544000000004E52465F75
:1020D0004552524F525F4E4F545F464F554E44004B
:1020E0004E52465F4552524F525F494E56414C49FF
:1020F000445F5354415445004E52465F4552524F3F
:10210000525F444154415F53495A45004E52465F25
:102110004552524F525F494F5F50454E44494E47DA
:10212000000000004E52465F4552524F525F5356D8
:10213000435F48414E444C45525F4D495353494ECD
:10214000470000004E52465F4552524F525F494E83
:1021500056414C49445F4C454E47544800000000EE
:102160004E52465F4552524F525F4452565F54574B
:10217000495F4552525F414E41434B004E52465FCC
:102180004552524F525F4452565F5457495F455231
:10219000525F444E41434B004E52465F4552524FB0
:1021A000525F494E5445524E414C00004E52465FDC
:1021B0004552524F525F53544F524147455F465527
:1021C0004C4C00004E52465F4552524F525F4E55A6
:1021D0004C4C00004E52465F4552524F525F494EA2
:1021E00056414C49445F504152414D004E52465F6A
:1021F0004552524F525F4E4F5F4D454D000000001B
:102200004E52465F4552524F525F464F52424944EA
:1022100044454E004E52465F4552524F525F445223
:10222000565F5457495F4552525F4F56455252557B
:102230004E0000004E52465F4552524F525F494E8B
:1022400056414C49445F4144445200004E52465F5F
:102250004552524F525F5245534F555243455300DA
:102260004E52465F4552524F525F494E56414C497D
:10227000445F464C414753004E52465F53554343DB
:10228000455353004E52465F4552524F525F424CA7
:10229000455F495053505F4348414E4E454C5F4166
:1022A0004C52454144595F4558495354530000002E
:1022B0004E52465F4552524F525F434F4E4E5F4320
:1022C0004F554E54000000004E52465F4552524F4B
:1022D000525F54494D454F55540000004E52465FE1
:1022E0004552524F525F4255535900007761726E0A
:1022F000696E670064656275670000001B5B313BB7
:1023000033306D001B5B306D000000001B5B313B08
:1023100033316D001B5B313B33326D001B5B313B56
:1023200033336D001B5B313B33346D001B5B313B42
:1023300033356D001B5B313B33366D001B5B313B2E
:1023400033376D00696E666F000000006572726F52
:102350007200000073645F626C655F6366675F7341
:10236000657428292072657475726E656420257302
:10237000207768656E20617474656D7074696E672E
:1023800020746F2073657420424C455F474154545C
:10239000535F4346475F534552564943455F434861
:1023A000414E4745442E000073645F626C655F6375
:1023B00066675F73657428292072657475726E652F
:1023C00064202573207768656E20617474656D7074
:1023D00074696E6720746F2073657420424C455F8A
:1023E000434F4D4D4F4E5F4346475F56535F5555E4
:1023F00049442E0073645F626C655F6366675F7358
:10240000657428292072657475726E656420257361
:10241000207768656E20617474656D7074696E678D
:1024200020746F2073657420424C455F47415454BB
:10243000535F4346475F415454525F5441425F5398
:10244000495A452E0000000073645F626C655F634B
:1024500066675F73657428292072657475726E658E
:1024600064202573207768656E20617474656D70D3
:1024700074696E6720746F2073657420424C455FE9
:10248000434F4E4E5F4346475F4741502E0000008A
:1024900073645F626C655F6366675F736574282948
:1024A0002072657475726E65642025732077686587
:1024B0006E20617474656D7074696E6720746F202E
:1024C00073657420424C455F4741505F4346475F08
:1024D000524F4C455F434F554E542E006E72665F0F
:1024E000626C655F6761747400000000636C6F6309
:1024F0006B000000434C4F434B0000004750494FD6
:1025000054450000505253005541525445000000BC
:1025100061746669666F2E6D5F7175657565000023
:102520006E72665F6673746F7261676500000000AB
:1025300061746669666F2E6D5F6669666F00000084
:102540007077725F6D676D740000000062616C6C83
:102550006F632E6C6F675F6D656D706F6F6C0000E1
:10256000617070006E72665F736468006E72665FA1
:102570007364685F626C65006E72665F7364685F47
:10258000736F6300B4260200481B0020F0010000B6
:102590002095010010270200381D0020E0140000E3
:1025A000D09A0100DC24020000000303EC240200A6
:1025B00000000000F424020000000000FC240200DF
:1025C00000000000042502000000000008250200B1
:1025D000000000001025020000000003202502007A
:1025E0000000030330250200000000034025020024
:1025F000000000004C2502000000000360250200DE
:102600000000030364250200000003036C250200A0
:10261000000003037825020000000303981C00203B
:10262000901C0020981C002034250020241D002030
:102630001800000005AA010000000000B5D3010049
:10264000381D00204BA30100541D002099A8010053
:102650000000000009A901000000000009AB010012
:1026600000000000DBD40100481D0020F1A701009C
:102670000000000069DA010000000000910E020075
:1026800000000000A1DA010000000000B5A3010075
:10269000541D00209DE701000000000029E9010011
:1026A00000000000610502000000000081DA010066
:1026B00000000000062BFFFF0A18010B2AF1FB2E79
:1026C000212A18017909390A016113141D024020D9
:1026D0000A1A1C44122042400425581D02144C239F
:1026E0000214EC22021A44081AF4081A04081AFC0C
:1026F000081A0C081A14041A1C041A24041A2C04AC
:102700001A34041A3C04518490D0030445B5BC012A
:040000050001920163
:00000001FF
